 xbdm

 Timestamp is 416ae404 (Mon Oct 11 21:50:28 2004)

 Preferred load address is 00400000

 Start         Length     Name                   Class
 0001:00000000 000001f0H .idata$5                CODE
 0001:000001f0 00001fbaH .rdata                  CODE
 0001:000021ac 00000047H .rdata$debug            CODE
 0001:00002200 0000fc6cH .text                   CODE
 0002:00000000 0000a065H XNET                    CODE
 0002:0000a068 0000018cH XNET_RD                 CODE
 0003:00000000 00000d38H .data                   DATA
 0003:00000d40 00002bacH .bss                    DATA
 0004:00000000 00000004H .tls$                   DATA
 0005:00000000 00000151H .edata                  DATA
 0006:00000000 00000014H .idata$2                CODE
 0006:00000014 00000014H .idata$3                CODE
 0006:00000028 000001f0H .idata$4                CODE
 0006:00000218 0000000eH .idata$6                CODE
 0007:00000000 00000010H .XBLD$A                 DATA
 0007:00000010 00000020H .XBLD$V                 DATA
 0008:00000000 00000058H .rsrc$01                DATA
 0008:00000060 00000320H .rsrc$02                DATA

  Address         Publics by Value              Rva+Base     Lib:Object

 0000:00000000       ___safe_se_handler_count   00000000     <absolute>
 0000:00000000       ___safe_se_handler_table   00000000     <absolute>
 0000:00000000       __except_list              00000000     <absolute>
 0001:00000000       __imp__ExSaveNonVolatileSetting@16 00400360     xboxkrnl:xboxkrnl.exe
 0001:00000004       __imp__MmCreateKernelStack@8 00400364     xboxkrnl:xboxkrnl.exe
 0001:00000008       __imp__RtlLeaveCriticalSection@4 00400368     xboxkrnl:xboxkrnl.exe
 0001:0000000c       __imp__NtReadFile@32       0040036c     xboxkrnl:xboxkrnl.exe
 0001:00000010       __imp__RtlEnterCriticalSection@4 00400370     xboxkrnl:xboxkrnl.exe
 0001:00000014       __imp__NtClose@4           00400374     xboxkrnl:xboxkrnl.exe
 0001:00000018       __imp__NtQueryDirectoryFile@40 00400378     xboxkrnl:xboxkrnl.exe
 0001:0000001c       __imp__NtWriteFile@32      0040037c     xboxkrnl:xboxkrnl.exe
 0001:00000020       __imp__MmDeleteKernelStack@8 00400380     xboxkrnl:xboxkrnl.exe
 0001:00000024       __imp_@ObfDereferenceObject@4 00400384     xboxkrnl:xboxkrnl.exe
 0001:00000028       __imp__DbgPrint            00400388     xboxkrnl:xboxkrnl.exe
 0001:0000002c       __imp__ObReferenceObjectByHandle@12 0040038c     xboxkrnl:xboxkrnl.exe
 0001:00000030       _PsThreadObjectType        00400390     xboxkrnl:xboxkrnl.exe
 0001:00000030       __imp__PsThreadObjectType  00400390     xboxkrnl:xboxkrnl.exe
 0001:00000034       __imp_@KfLowerIrql@4       00400394     xboxkrnl:xboxkrnl.exe
 0001:00000038       __imp__KeRaiseIrqlToDpcLevel@0 00400398     xboxkrnl:xboxkrnl.exe
 0001:0000003c       __imp__KeWaitForSingleObject@20 0040039c     xboxkrnl:xboxkrnl.exe
 0001:00000040       __imp__PsSetCreateThreadNotifyRoutine@4 004003a0     xboxkrnl:xboxkrnl.exe
 0001:00000044       __imp__HalRegisterShutdownNotification@8 004003a4     xboxkrnl:xboxkrnl.exe
 0001:00000048       __imp__RtlInitializeCriticalSection@4 004003a8     xboxkrnl:xboxkrnl.exe
 0001:0000004c       __imp__KeAlertThread@8     004003ac     xboxkrnl:xboxkrnl.exe
 0001:00000050       __imp__KeQuerySystemTime@4 004003b0     xboxkrnl:xboxkrnl.exe
 0001:00000054       __imp__KeSetEvent@12       004003b4     xboxkrnl:xboxkrnl.exe
 0001:00000058       __imp__KeSetBasePriorityThread@8 004003b8     xboxkrnl:xboxkrnl.exe
 0001:0000005c       __imp__PsCreateSystemThread@20 004003bc     xboxkrnl:xboxkrnl.exe
 0001:00000060       __imp_@ObfReferenceObject@4 004003c0     xboxkrnl:xboxkrnl.exe
 0001:00000064       __imp__KdDebuggerEnabled   004003c4     xboxkrnl:xboxkrnl.exe
 0001:00000064       _KdDebuggerEnabled         004003c4     xboxkrnl:xboxkrnl.exe
 0001:00000068       __imp__NtOpenFile@24       004003c8     xboxkrnl:xboxkrnl.exe
 0001:0000006c       __imp__RtlInitAnsiString@8 004003cc     xboxkrnl:xboxkrnl.exe
 0001:00000070       __imp__NtSetInformationFile@20 004003d0     xboxkrnl:xboxkrnl.exe
 0001:00000074       __imp__NtQueryInformationFile@20 004003d4     xboxkrnl:xboxkrnl.exe
 0001:00000078       __imp__NtQueryFullAttributesFile@8 004003d8     xboxkrnl:xboxkrnl.exe
 0001:0000007c       __imp__NtCreateFile@36     004003dc     xboxkrnl:xboxkrnl.exe
 0001:00000080       __imp__MmIsAddressValid@4  004003e0     xboxkrnl:xboxkrnl.exe
 0001:00000084       __imp__ExQueryNonVolatileSetting@20 004003e4     xboxkrnl:xboxkrnl.exe
 0001:00000088       __imp__NtSetSystemTime@8   004003e8     xboxkrnl:xboxkrnl.exe
 0001:0000008c       __imp__MmAllocateSystemMemory@8 004003ec     xboxkrnl:xboxkrnl.exe
 0001:00000090       __imp__MmFreeSystemMemory@8 004003f0     xboxkrnl:xboxkrnl.exe
 0001:00000094       __imp__NtQueryDirectoryObject@24 004003f4     xboxkrnl:xboxkrnl.exe
 0001:00000098       __imp__NtOpenDirectoryObject@8 004003f8     xboxkrnl:xboxkrnl.exe
 0001:0000009c       __imp__NtQueryVolumeInformationFile@20 004003fc     xboxkrnl:xboxkrnl.exe
 0001:000000a0       __imp__KeTickCount         00400400     xboxkrnl:xboxkrnl.exe
 0001:000000a0       _KeTickCount               00400400     xboxkrnl:xboxkrnl.exe
 0001:000000a4       __imp__XcModExp@20         00400404     xboxkrnl:xboxkrnl.exe
 0001:000000a8       __imp__HalReadWritePCISpace@24 00400408     xboxkrnl:xboxkrnl.exe
 0001:000000ac       __imp__MmQueryStatistics@4 0040040c     xboxkrnl:xboxkrnl.exe
 0001:000000b0       __imp__MmGlobalData        00400410     xboxkrnl:xboxkrnl.exe
 0001:000000b0       _MmGlobalData              00400410     xboxkrnl:xboxkrnl.exe
 0001:000000b4       __imp__IoSynchronousFsdRequest@20 00400414     xboxkrnl:xboxkrnl.exe
 0001:000000b8       __imp__ObReferenceObjectByName@20 00400418     xboxkrnl:xboxkrnl.exe
 0001:000000bc       __imp__IoDeviceObjectType  0040041c     xboxkrnl:xboxkrnl.exe
 0001:000000bc       _IoDeviceObjectType        0040041c     xboxkrnl:xboxkrnl.exe
 0001:000000c0       __imp__NtResumeThread@8    00400420     xboxkrnl:xboxkrnl.exe
 0001:000000c4       __imp__NtCreateDirectoryObject@8 00400424     xboxkrnl:xboxkrnl.exe
 0001:000000c8       __imp__ObOpenObjectByName@16 00400428     xboxkrnl:xboxkrnl.exe
 0001:000000cc       __imp__ObInsertObject@16   0040042c     xboxkrnl:xboxkrnl.exe
 0001:000000d0       __imp__ObCreateObject@16   00400430     xboxkrnl:xboxkrnl.exe
 0001:000000d4       __imp__ObMakeTemporaryObject@4 00400434     xboxkrnl:xboxkrnl.exe
 0001:000000d8       __imp_@HalRequestSoftwareInterrupt@4 00400438     xboxkrnl:xboxkrnl.exe
 0001:000000dc       __imp__KeResetEvent@4      0040043c     xboxkrnl:xboxkrnl.exe
 0001:000000e0       __imp_@KfRaiseIrql@4       00400440     xboxkrnl:xboxkrnl.exe
 0001:000000e4       __imp__KeInsertQueueDpc@12 00400444     xboxkrnl:xboxkrnl.exe
 0001:000000e8       _KdDebuggerNotPresent      00400448     xboxkrnl:xboxkrnl.exe
 0001:000000e8       __imp__KdDebuggerNotPresent 00400448     xboxkrnl:xboxkrnl.exe
 0001:000000ec       __imp__KeInitializeDpc@12  0040044c     xboxkrnl:xboxkrnl.exe
 0001:000000f0       __imp__MmDbgReleaseAddress@8 00400450     xboxkrnl:xboxkrnl.exe
 0001:000000f4       __imp__MmDbgWriteCheck@8   00400454     xboxkrnl:xboxkrnl.exe
 0001:000000f8       __imp__KeSuspendThread@4   00400458     xboxkrnl:xboxkrnl.exe
 0001:000000fc       __imp__KeResumeThread@4    0040045c     xboxkrnl:xboxkrnl.exe
 0001:00000100       __imp__KeBugCheck@4        00400460     xboxkrnl:xboxkrnl.exe
 0001:00000104       __imp__HalReturnToFirmware@4 00400464     xboxkrnl:xboxkrnl.exe
 0001:00000108       __imp__XeImageFileName     00400468     xboxkrnl:xboxkrnl.exe
 0001:00000108       _XeImageFileName           00400468     xboxkrnl:xboxkrnl.exe
 0001:0000010c       __imp__DbgLoadImageSymbols@12 0040046c     xboxkrnl:xboxkrnl.exe
 0001:00000110       __imp_@ExfInterlockedInsertTailList@8 00400470     xboxkrnl:xboxkrnl.exe
 0001:00000114       __imp__RtlAnsiStringToUnicodeString@12 00400474     xboxkrnl:xboxkrnl.exe
 0001:00000118       __imp__MmDbgFreeMemory@8   00400478     xboxkrnl:xboxkrnl.exe
 0001:0000011c       __imp__DbgUnLoadImageSymbols@12 0040047c     xboxkrnl:xboxkrnl.exe
 0001:00000120       __imp__RtlUnicodeStringToAnsiString@12 00400480     xboxkrnl:xboxkrnl.exe
 0001:00000124       __imp__ExFreePool@4        00400484     xboxkrnl:xboxkrnl.exe
 0001:00000128       __imp__ExAllocatePoolWithTag@8 00400488     xboxkrnl:xboxkrnl.exe
 0001:0000012c       __imp__ExAllocatePool@4    0040048c     xboxkrnl:xboxkrnl.exe
 0001:00000130       __imp__MmDbgAllocateMemory@8 00400490     xboxkrnl:xboxkrnl.exe
 0001:00000134       _KeTimeIncrement           00400494     xboxkrnl:xboxkrnl.exe
 0001:00000134       __imp__KeTimeIncrement     00400494     xboxkrnl:xboxkrnl.exe
 0001:00000138       __imp__KeSetTimerEx@20     00400498     xboxkrnl:xboxkrnl.exe
 0001:0000013c       __imp__KeInitializeTimerEx@8 0040049c     xboxkrnl:xboxkrnl.exe
 0001:00000140       __imp__ObOpenObjectByPointer@12 004004a0     xboxkrnl:xboxkrnl.exe
 0001:00000144       __imp__RtlFillMemoryUlong@12 004004a4     xboxkrnl:xboxkrnl.exe
 0001:00000148       __imp_@InterlockedPushEntrySList@8 004004a8     xboxkrnl:xboxkrnl.exe
 0001:0000014c       __imp__KeBugCheckEx@20     004004ac     xboxkrnl:xboxkrnl.exe
 0001:00000150       __imp_@InterlockedPopEntrySList@4 004004b0     xboxkrnl:xboxkrnl.exe
 0001:00000154       __imp__RtlNtStatusToDosError@4 004004b4     xboxkrnl:xboxkrnl.exe
 0001:00000158       __imp__KeDelayExecutionThread@12 004004b8     xboxkrnl:xboxkrnl.exe
 0001:0000015c       __imp__PsTerminateSystemThread@4 004004bc     xboxkrnl:xboxkrnl.exe
 0001:00000160       __imp__PsCreateSystemThreadEx@40 004004c0     xboxkrnl:xboxkrnl.exe
 0001:00000164       __imp__KeStallExecutionProcessor@4 004004c4     xboxkrnl:xboxkrnl.exe
 0001:00000168       __imp__MmUnmapIoSpace@8    004004c8     xboxkrnl:xboxkrnl.exe
 0001:0000016c       __imp__MmMapIoSpace@12     004004cc     xboxkrnl:xboxkrnl.exe
 0001:00000170       __imp__ExEventObjectType   004004d0     xboxkrnl:xboxkrnl.exe
 0001:00000170       _ExEventObjectType         004004d0     xboxkrnl:xboxkrnl.exe
 0001:00000174       __imp__KeWaitForMultipleObjects@32 004004d4     xboxkrnl:xboxkrnl.exe
 0001:00000178       __imp__PhyGetLinkState@4   004004d8     xboxkrnl:xboxkrnl.exe
 0001:0000017c       __imp__PhyInitialize@8     004004dc     xboxkrnl:xboxkrnl.exe
 0001:00000180       __imp__XcRC4Crypt@12       004004e0     xboxkrnl:xboxkrnl.exe
 0001:00000184       __imp__XcRC4Key@12         004004e4     xboxkrnl:xboxkrnl.exe
 0001:00000188       __imp__XcSHAFinal@8        004004e8     xboxkrnl:xboxkrnl.exe
 0001:0000018c       __imp__XcSHAUpdate@12      004004ec     xboxkrnl:xboxkrnl.exe
 0001:00000190       __imp__XcSHAInit@4         004004f0     xboxkrnl:xboxkrnl.exe
 0001:00000194       __imp__KeRemoveQueueDpc@4  004004f4     xboxkrnl:xboxkrnl.exe
 0001:00000198       __imp__KeCancelTimer@4     004004f8     xboxkrnl:xboxkrnl.exe
 0001:0000019c       _HalDiskSerialNumber       004004fc     xboxkrnl:xboxkrnl.exe
 0001:0000019c       __imp__HalDiskSerialNumber 004004fc     xboxkrnl:xboxkrnl.exe
 0001:000001a0       _HalDiskModelNumber        00400500     xboxkrnl:xboxkrnl.exe
 0001:000001a0       __imp__HalDiskModelNumber  00400500     xboxkrnl:xboxkrnl.exe
 0001:000001a4       __imp__XcBlockCryptCBC@28  00400504     xboxkrnl:xboxkrnl.exe
 0001:000001a8       __imp__XcKeyTable@12       00400508     xboxkrnl:xboxkrnl.exe
 0001:000001ac       __imp__XcDESKeyParity@8    0040050c     xboxkrnl:xboxkrnl.exe
 0001:000001b0       __imp__XcHMAC@28           00400510     xboxkrnl:xboxkrnl.exe
 0001:000001b4       __imp__MmAllocateContiguousMemoryEx@20 00400514     xboxkrnl:xboxkrnl.exe
 0001:000001b8       __imp__MmFreeContiguousMemory@4 00400518     xboxkrnl:xboxkrnl.exe
 0001:000001bc       __imp__MmLockUnlockBufferPages@12 0040051c     xboxkrnl:xboxkrnl.exe
 0001:000001c0       __imp__MmGetPhysicalAddress@4 00400520     xboxkrnl:xboxkrnl.exe
 0001:000001c4       __imp__KeDisconnectInterrupt@4 00400524     xboxkrnl:xboxkrnl.exe
 0001:000001c8       __imp__KeConnectInterrupt@4 00400528     xboxkrnl:xboxkrnl.exe
 0001:000001cc       __imp__KeInitializeInterrupt@28 0040052c     xboxkrnl:xboxkrnl.exe
 0001:000001d0       __imp__HalGetInterruptVector@8 00400530     xboxkrnl:xboxkrnl.exe
 0001:000001d4       __imp__MmPersistContiguousMemory@12 00400534     xboxkrnl:xboxkrnl.exe
 0001:000001d8       __imp__MmAllocateContiguousMemory@4 00400538     xboxkrnl:xboxkrnl.exe
 0001:000001dc       __imp__LaunchDataPage      0040053c     xboxkrnl:xboxkrnl.exe
 0001:000001dc       _LaunchDataPage            0040053c     xboxkrnl:xboxkrnl.exe
 0001:000001e0       __imp__NtFsControlFile@40  00400540     xboxkrnl:xboxkrnl.exe
 0001:000001e4       __imp__NtDeviceIoControlFile@40 00400544     xboxkrnl:xboxkrnl.exe
 0001:000001e8       __imp__RtlUnwind@16        00400548     xboxkrnl:xboxkrnl.exe
 0001:000001ec       \177xboxkrnl_NULL_THUNK_DATA 0040054c     xboxkrnl:xboxkrnl.exe
 0001:0000020c       ??_C@_04HLBMEOMD@addr?$AA@ 0040056c     dminit.obj
 0001:00000214       ??_C@_08JADIEHCF@staticip?$AA@ 00400574     dminit.obj
 0001:00000220       ??_C@_08LBEDNJME@notifyat?$AA@ 00400580     dminit.obj
 0001:0000022c       ??_C@_06LIGDCBBN@notify?$AA@ 0040058c     dminit.obj
 0001:00000234       ??_C@_04PEGFANN@stop?$AA@  00400594     dminit.obj
 0001:0000023c       ??_C@_07PLNOAMKO@forever?$AA@ 0040059c     dminit.obj
 0001:00000244       ??_C@_04PNOAOIAG@wait?$AA@ 004005a4     dminit.obj
 0001:0000024c       ??_C@_08LKAPKLCD@?$CFs?2?$CF?$CK?4?$CKs?$AA@ 004005ac     dminit.obj
 0001:00000258       ??_C@_02PCIJFNDE@?$AN?6?$AA@ 004005b8     dminit.obj
 0001:0000025c       ??_C@_0BF@ENMDJCFG@staticip?5addr?$DN0x?$CF08x?$AA@ 004005bc     dminit.obj
 0001:00000274       ??_C@_0O@DEFJBBCE@dbgname?5name?$DN?$AA@ 004005d4     dminit.obj
 0001:00000284       ??_C@_0N@LDDCMAAC@wait?5forever?$AA@ 004005e4     dminit.obj
 0001:00000294       ??_C@_09KFEMIOCO@wait?5stop?$AA@ 004005f4     dminit.obj
 0001:000002a0       ??_C@_06LMJMCNHD@?$FLxbdm?$FN?$AA@ 00400600     dminit.obj
 0001:000002a8       ??_C@_0BO@DBMCNND@dm?3?5could?5not?5get?5new?5thread?6?$AA@ 00400608     dminit.obj
 0001:000002c8       ??_C@_0CB@CCMKOGFJ@dm?3?5could?5not?5alloc?5thread?5data?6@ 00400628     dminit.obj
 0001:000002ec       ??_C@_0CF@PBEGCFCL@dm?3?5waiting?5for?5debugger?5connect@ 0040064c     dminit.obj
 0001:00000314       ??_C@_07GDJNMEFM@xtlinfo?$AA@ 00400674     dmserv.obj
 0001:0000031c       ??_C@_07EAJMDMGA@xbeinfo?$AA@ 0040067c     dmserv.obj
 0001:00000324       ??_C@_06GDDMHIDB@vssnap?$AA@ 00400684     dmserv.obj
 0001:0000032c       ??_C@_08BJHBHMAO@userlist?$AA@ 0040068c     dmserv.obj
 0001:00000338       ??_C@_04CCHAHKJA@user?$AA@ 00400698     dmserv.obj
 0001:00000340       ??_C@_05PHLGJONK@title?$AA@ 004006a0     dmserv.obj
 0001:00000348       ??_C@_07NFPADACG@threads?$AA@ 004006a8     dmserv.obj
 0001:00000350       ??_C@_0L@BKNDBIB@threadinfo?$AA@ 004006b0     dmserv.obj
 0001:0000035c       ??_C@_07FOLNGFGF@systime?$AA@ 004006bc     dmserv.obj
 0001:00000364       ??_C@_0L@BPAFCKOI@sysfileupd?$AA@ 004006c4     dmserv.obj
 0001:00000370       ??_C@_07DNBGJJHB@suspend?$AA@ 004006d0     dmserv.obj
 0001:00000378       ??_C@_06OHAICPNE@stopon?$AA@ 004006d8     dmserv.obj
 0001:00000380       ??_C@_0M@INHAMGK@setuserpriv?$AA@ 004006e0     dmserv.obj
 0001:0000038c       ??_C@_0L@KNFJGCPP@setsystime?$AA@ 004006ec     dmserv.obj
 0001:00000398       ??_C@_06LMHLABCO@setmem?$AA@ 004006f8     dmserv.obj
 0001:000003a0       ??_C@_0BC@LIFABAIC@setfileattributes?$AA@ 00400700     dmserv.obj
 0001:000003b4       ??_C@_0L@GJEGBGFG@setcontext?$AA@ 00400714     dmserv.obj
 0001:000003c0       ??_C@_09CJOMHFFI@setconfig?$AA@ 00400720     dmserv.obj
 0001:000003cc       ??_C@_08JCEFHKI@sendfile?$AA@ 0040072c     dmserv.obj
 0001:000003d8       ??_C@_0L@CMHOPIGK@screenshot?$AA@ 00400738     dmserv.obj
 0001:000003e4       ??_C@_06PLELHCEK@resume?$AA@ 00400744     dmserv.obj
 0001:000003ec       ??_C@_06LMEAOBLB@rename?$AA@ 0040074c     dmserv.obj
 0001:000003f4       ??_C@_06MJDCIMPN@reboot?$AA@ 00400754     dmserv.obj
 0001:000003fc       ??_C@_07JDEKNMHA@querypc?$AA@ 0040075c     dmserv.obj
 0001:00000404       ??_C@_06OMENAL@pssnap?$AA@ 00400764     dmserv.obj
 0001:0000040c       ??_C@_06HJDMFGA@pclist?$AA@ 0040076c     dmserv.obj
 0001:00000414       ??_C@_08BAHAMCF@nostopon?$AA@ 00400774     dmserv.obj
 0001:00000420       ??_C@_07DFGEOAEG@modules?$AA@ 00400780     dmserv.obj
 0001:00000428       ??_C@_0M@ODADOEJE@modsections?$AA@ 00400788     dmserv.obj
 0001:00000434       ??_C@_07GINKICOP@modlong?$AA@ 00400794     dmserv.obj
 0001:0000043c       ??_C@_08MEADNPCK@mmglobal?$AA@ 0040079c     dmserv.obj
 0001:00000448       ??_C@_05PKPOIPAL@mkdir?$AA@ 004007a8     dmserv.obj
 0001:00000450       ??_C@_09LBHLKDFJ@magicboot?$AA@ 004007b0     dmserv.obj
 0001:0000045c       ??_C@_08CHLECKKA@lockmode?$AA@ 004007bc     dmserv.obj
 0001:00000468       ??_C@_07GOLGDHCL@keyxchg?$AA@ 004007c8     dmserv.obj
 0001:00000470       ??_C@_02EFKNKMIP@kd?$AA@   004007d0     dmserv.obj
 0001:00000474       ??_C@_09OGJDHPNM@isstopped?$AA@ 004007d4     dmserv.obj
 0001:00000480       ??_C@_07INDDFIAE@isbreak?$AA@ 004007e0     dmserv.obj
 0001:00000488       ??_C@_08LEPLIKMH@irtsweep?$AA@ 004007e8     dmserv.obj
 0001:00000494       ??_C@_04BJJLCKLO@halt?$AA@ 004007f4     dmserv.obj
 0001:0000049c       ??_C@_08PDANPODO@gpucount?$AA@ 004007fc     dmserv.obj
 0001:000004a8       ??_C@_02KPEDIMCA@go?$AA@   00400808     dmserv.obj
 0001:000004ac       ??_C@_0M@HMJNKOJ@getuserpriv?$AA@ 0040080c     dmserv.obj
 0001:000004b8       ??_C@_06CPOKLJPD@getmem?$AA@ 00400818     dmserv.obj
 0001:000004c0       ??_C@_0BC@JNFLJLJM@getfileattributes?$AA@ 00400820     dmserv.obj
 0001:000004d4       ??_C@_07NFDCGD@getfile?$AA@ 00400834     dmserv.obj
 0001:000004dc       ??_C@_0O@JKOJCMIC@getextcontext?$AA@ 0040083c     dmserv.obj
 0001:000004ec       ??_C@_0L@HHGJKBBP@getcontext?$AA@ 0040084c     dmserv.obj
 0001:000004f8       ??_C@_08FCFLENND@funccall?$AA@ 00400858     dmserv.obj
 0001:00000504       ??_C@_06COMGLGOP@fmtfat?$AA@ 00400864     dmserv.obj
 0001:0000050c       ??_C@_05LEFLIPJH@flash?$AA@ 0040086c     dmserv.obj
 0001:00000514       ??_C@_06PKEIMIIG@dvdblk?$AA@ 00400874     dmserv.obj
 0001:0000051c       ??_C@_09FABFAIG@drivelist?$AA@ 0040087c     dmserv.obj
 0001:00000528       ??_C@_0P@GODBNCAM@drivefreespace?$AA@ 00400888     dmserv.obj
 0001:00000538       ??_C@_07JBLAGDBF@dirlist?$AA@ 00400898     dmserv.obj
 0001:00000540       ??_C@_06FOBLBEIN@delete?$AA@ 004008a0     dmserv.obj
 0001:00000548       ??_C@_08NBJPCMHP@deftitle?$AA@ 004008a8     dmserv.obj
 0001:00000554       ??_C@_08MGAKGBNH@dedicate?$AA@ 004008b4     dmserv.obj
 0001:00000560       ??_C@_09LOFBDIHH@debugmode?$AA@ 004008c0     dmserv.obj
 0001:0000056c       ??_C@_08BJECCCMA@debugger?$AA@ 004008cc     dmserv.obj
 0001:00000578       ??_C@_07DKLJHCCC@dbgname?$AA@ 004008d8     dmserv.obj
 0001:00000580       ??_C@_08DLICDMBN@continue?$AA@ 004008e0     dmserv.obj
 0001:0000058c       ??_C@_0L@MFALGBGB@capcontrol?$AA@ 004008ec     dmserv.obj
 0001:00000598       ??_C@_03MDONDFG@bye?$AA@   004008f8     dmserv.obj
 0001:0000059c       ??_C@_05ELPHFHOI@break?$AA@ 004008fc     dmserv.obj
 0001:000005a4       ??_C@_05PIHPMGOO@boxid?$AA@ 00400904     dmserv.obj
 0001:000005ac       ??_C@_08FBHDOKDP@authuser?$AA@ 0040090c     dmserv.obj
 0001:000005b8       ??_C@_07BIPIKPNE@altaddr?$AA@ 00400918     dmserv.obj
 0001:000005c0       ??_C@_07DGFLOGKM@adminpw?$AA@ 00400920     dmserv.obj
 0001:000005c8       ??_C@_0M@CGENBBIN@Cr0NpxState?$AA@ 00400928     dmserv.obj
 0001:000005d4       ??_C@_03JAPJIOAL@Esi?$AA@  00400934     dmserv.obj
 0001:000005d8       ??_C@_03IJJADLPO@Edi?$AA@  00400938     dmserv.obj
 0001:000005dc       ??_C@_03NKEJBIOO@Edx?$AA@  0040093c     dmserv.obj
 0001:000005e0       ??_C@_03NPAGAOGL@Ecx?$AA@  00400940     dmserv.obj
 0001:000005e4       ??_C@_03NOMEGEFM@Ebx?$AA@  00400944     dmserv.obj
 0001:000005e8       ??_C@_03NMICNKAF@Eax?$AA@  00400948     dmserv.obj
 0001:000005ec       ??_C@_06DLHDGOJE@EFlags?$AA@ 0040094c     dmserv.obj
 0001:000005f4       ??_C@_03BKEIABLF@Eip?$AA@  00400954     dmserv.obj
 0001:000005f8       ??_C@_03LPJCHBD@Esp?$AA@   00400958     dmserv.obj
 0001:000005fc       ??_C@_03BGBNOOFE@Ebp?$AA@  0040095c     dmserv.obj
 0001:00000600       _rgchHex                   00400960     dmserv.obj
 0001:00000614       ??_C@_0M@PCENNPGA@?$CFd?4?$CFd?4?$CFd?4?$CFd?$AA@ 00400974     dmserv.obj
 0001:00000620       ??_C@_0BC@PFIFDHBI@?$CFs?$DL?$CFs?$DL?$CFs?$DL?$CFd?$DL?$CFd?$AN?6?$AA?$AA@ 00400980     dmserv.obj
 0001:00000634       ??_C@_07BOHFNJFC@heyhey?$CB?$AA@ 00400994     dmserv.obj
 0001:0000063c       ??_C@_04MFDNODIH@xbox?$AA@ 0040099c     dmserv.obj
 0001:00000644       ??_C@_04OONEELOO@ping?$AA@ 004009a4     dmserv.obj
 0001:0000064c       ??_C@_0O@JHGCPJGI@192?4168?41?4102?$AA@ 004009ac     dmserv.obj
 0001:0000065c       ??_C@_0L@FEFPBOLE@missing?5?$CFs?$AA@ 004009bc     dmserv.obj
 0001:00000668       ??_C@_0BO@BEGMHLED@dedicated?5connection?5required?$AA@ 004009c8     dmserv.obj
 0001:00000688       ??_C@_02GIPFHKNO@OK?$AA@   004009e8     dmserv.obj
 0001:0000068c       ??_C@_0BL@JOELFKAM@multiline?5response?5follows?$AA@ 004009ec     dmserv.obj
 0001:000006a8       ??_C@_0BI@BLHJFM@binary?5response?5follows?$AA@ 00400a08     dmserv.obj
 0001:000006c0       ??_C@_0BB@PALNPLNJ@send?5binary?5data?$AA@ 00400a20     dmserv.obj
 0001:000006d1       ??_C@_00CNPNBAHC@?$AA@     00400a31     dmserv.obj
 0001:000006d4       ??_C@_0BG@OMIDBPHK@key?5exchange?5required?$AA@ 00400a34     dmserv.obj
 0001:000006ec       ??_C@_0O@NHKHFJHK@access?5denied?$AA@ 00400a4c     dmserv.obj
 0001:000006fc       ??_C@_0BC@KBHHJOIK@no?5room?5on?5device?$AA@ 00400a5c     dmserv.obj
 0001:00000710       ??_C@_0P@EJGIMKLJ@not?5debuggable?$AA@ 00400a70     dmserv.obj
 0001:00000720       ??_C@_0N@CCFLCBNA@type?5invalid?$AA@ 00400a80     dmserv.obj
 0001:00000730       ??_C@_0BD@MEDAILKF@data?5not?5available?$AA@ 00400a90     dmserv.obj
 0001:00000744       ??_C@_0BC@GIFDANAM@box?5is?5not?5locked?$AA@ 00400aa4     dmserv.obj
 0001:00000758       ??_C@_0BH@MFDCHBCM@file?5cannot?5be?5created?$AA@ 00400ab8     dmserv.obj
 0001:00000770       ??_C@_0BA@NINGALLD@unknown?5command?$AA@ 00400ad0     dmserv.obj
 0001:00000780       ??_C@_0M@OFAMHLMG@not?5stopped?$AA@ 00400ae0     dmserv.obj
 0001:0000078c       ??_C@_0BE@HKILNGAG@file?5must?5be?5copied?$AA@ 00400aec     dmserv.obj
 0001:000007a0       ??_C@_0BE@NKKNMLBF@file?5already?5exists?$AA@ 00400b00     dmserv.obj
 0001:000007b4       ??_C@_0BE@JIDOCPHM@directory?5not?5empty?$AA@ 00400b14     dmserv.obj
 0001:000007c8       ??_C@_0BE@KOACJCFI@filename?5is?5invalid?$AA@ 00400b28     dmserv.obj
 0001:000007dc       ??_C@_0P@CNAEEAKN@no?5such?5thread?$AA@ 00400b3c     dmserv.obj
 0001:000007ec       ??_C@_0BB@OCKADCMD@unexpected?5error?$AA@ 00400b4c     dmserv.obj
 0001:00000800       ??_C@_0O@BNNCBLEN@out?5of?5memory?$AA@ 00400b60     dmserv.obj
 0001:00000810       ??_C@_0O@BBEPBGMJ@bad?5parameter?$AA@ 00400b70     dmserv.obj
 0001:00000820       ??_C@_0P@LJOCCCLG@file?5not?5found?$AA@ 00400b80     dmserv.obj
 0001:00000830       ??_C@_0P@GMDNDOKH@no?5such?5module?$AA@ 00400b90     dmserv.obj
 0001:00000840       ??_C@_0BC@IBPNBLPK@memory?5not?5mapped?$AA@ 00400ba0     dmserv.obj
 0001:00000854       ??_C@_01LFCBOECM@?4?$AA@   00400bb4     dmserv.obj
 0001:00000858       ??_C@_0BD@ILJNLONI@406?9?5line?5too?5long?$AA@ 00400bb8     dmserv.obj
 0001:0000086c       ??_C@_0P@LHKPLOGH@201?9?5connected?$AA@ 00400bcc     dmserv.obj
 0001:0000087c       ??_C@_0CH@NCFCMBID@201?9?5boxid?$DN0q?$CF08x?$CF08x?5nonce?$DN0q?$CF0@ 00400bdc     dmserv.obj
 0001:000008a4       ??_C@_0CI@OLPEBHIE@401?9?5max?5number?5of?5connections?5e@ 00400c04     dmserv.obj
 0001:000008cc       ??_C@_08JMOJDPHD@200?9?5bye?$AA@ 00400c2c     dmserv.obj
 0001:000008d8       ??_C@_04MEMAJGDJ@name?$AA@ 00400c38     dmserv.obj
 0001:000008e0       ??_C@_07DBNODEFN@disable?$AA@ 00400c40     dmserv.obj
 0001:000008e8       ??_C@_06OFNJOBDK@enable?$AA@ 00400c48     dmserv.obj
 0001:000008f0       ??_C@_0BB@HDACDACL@improper?5command?$AA@ 00400c50     dmserv.obj
 0001:00000904       ??_C@_08PLPOIGIE@exceptif?$AA@ 00400c64     dmserv.obj
 0001:00000910       ??_C@_06JBKEBCGB@except?$AA@ 00400c70     dmserv.obj
 0001:00000918       ??_C@_0M@HPDGKBHD@kd?5disabled?$AA@ 00400c78     dmserv.obj
 0001:00000924       ??_C@_0L@OANFPHKA@kd?5enabled?$AA@ 00400c84     dmserv.obj
 0001:00000930       ??_C@_0BM@OBNGNCAI@notification?5limit?5exceeded?$AA@ 00400c90     dmserv.obj
 0001:0000094c       ??_C@_0N@JKMPLLJB@createthread?$AA@ 00400cac     dmserv.obj
 0001:0000095c       ??_C@_08NLNNCLEP@debugstr?$AA@ 00400cbc     dmserv.obj
 0001:00000968       ??_C@_03JCONGCKH@fce?$AA@  00400cc8     dmserv.obj
 0001:0000096c       ??_C@_0N@KNAHKBFB@stop?5on?5none?$AA@ 00400ccc     dmserv.obj
 0001:0000097c       ??_C@_0M@DFOCEODA@stop?5on?5all?$AA@ 00400cdc     dmserv.obj
 0001:00000988       ??_C@_03NFKEKGGK@all?$AA@  00400ce8     dmserv.obj
 0001:0000098c       ??_C@_0BA@FOBGILMN@already?5stopped?$AA@ 00400cec     dmserv.obj
 0001:0000099c       ??_C@_0M@KCKKNKEF@default?4xbe?$AA@ 00400cfc     dmserv.obj
 0001:000009a8       ??_C@_06IJDLPEM@length?$AA@ 00400d08     dmserv.obj
 0001:000009b0       ??_C@_0N@PHBADDFN@missing?5name?$AA@ 00400d10     dmserv.obj
 0001:000009c0       ??_C@_0BA@MFBJLJNL@file?5is?5too?5big?$AA@ 00400d20     dmserv.obj
 0001:000009d0       ??_C@_0FO@FGLICPJN@sizehi?$DN0x?$CFx?5sizelo?$DN0x?$CFx?5createhi@ 00400d30     dmserv.obj
 0001:00000a30       ??_C@_0L@EFCMAFLB@?5directory?$AA@ 00400d90     dmserv.obj
 0001:00000a3c       ??_C@_09NEHJELJP@?5readonly?$AA@ 00400d9c     dmserv.obj
 0001:00000a48       ??_C@_07JJJNOAOL@?5hidden?$AA@ 00400da8     dmserv.obj
 0001:00000a50       ??_C@_08OEGLCNAF@changelo?$AA@ 00400db0     dmserv.obj
 0001:00000a5c       ??_C@_08LFDICCFP@changehi?$AA@ 00400dbc     dmserv.obj
 0001:00000a68       ??_C@_08CLEJHLHC@createlo?$AA@ 00400dc8     dmserv.obj
 0001:00000a74       ??_C@_08HKBKHECI@createhi?$AA@ 00400dd4     dmserv.obj
 0001:00000a80       ??_C@_06JIKFICKK@hidden?$AA@ 00400de0     dmserv.obj
 0001:00000a88       ??_C@_08JOKHDEJH@readonly?$AA@ 00400de8     dmserv.obj
 0001:00000a94       ??_C@_0BI@NICIBCIC@new?5name?5does?5not?5exist?$AA@ 00400df4     dmserv.obj
 0001:00000aac       ??_C@_0BB@JDDNDBCG@missing?5new?5name?$AA@ 00400e0c     dmserv.obj
 0001:00000ac0       ??_C@_07GNAIFCPP@newname?$AA@ 00400e20     dmserv.obj
 0001:00000ac8       ??_C@_0P@FLLDBIDK@is?5a?5directory?$AA@ 00400e28     dmserv.obj
 0001:00000ad8       ??_C@_0BA@DOCPFFJG@not?5a?5directory?$AA@ 00400e38     dmserv.obj
 0001:00000ae8       ??_C@_03DAPAKLGM@dir?$AA@  00400e48     dmserv.obj
 0001:00000aec       ??_C@_06JMOJEPOI@name?$DN?$CC?$AA@ 00400e4c     dmserv.obj
 0001:00000af4       ??_C@_0BB@FHEJDJHB@unable?5to?5format?$AA@ 00400e54     dmserv.obj
 0001:00000b08       ??_C@_0BO@HNBKKHNC@?2Device?2Harddisk0?2Partition?$CFd?$AA@ 00400e68     dmserv.obj
 0001:00000b28       ??_C@_09IKAEIPAD@partition?$AA@ 00400e88     dmserv.obj
 0001:00000b34       ??_C@_07PNJCLMKK@cmdline?$AA@ 00400e94     dmserv.obj
 0001:00000b3c       ??_C@_0M@ODEICKAB@missing?5dir?$AA@ 00400e9c     dmserv.obj
 0001:00000b48       ??_C@_08EAFLGIKM@launcher?$AA@ 00400ea8     dmserv.obj
 0001:00000b54       ??_C@_04CGFJFPFD@none?$AA@ 00400eb4     dmserv.obj
 0001:00000b5c       ??_C@_0BE@IJAHOKJO@memory?5data?5follows?$AA@ 00400ebc     dmserv.obj
 0001:00000b70       ??_C@_0BK@NEHGJNBJ@400?9?5syntax?5error?5in?5data?$AA@ 00400ed0     dmserv.obj
 0001:00000b8c       ??_C@_0N@KDFPIGF@set?5?$CFd?5bytes?$AA@ 00400eec     dmserv.obj
 0001:00000b9c       ??_C@_04PJOLNDGD@data?$AA@ 00400efc     dmserv.obj
 0001:00000ba4       ??_C@_04HGIPLDBL@?$CFd?$AN?6?$AA@ 00400f04     dmserv.obj
 0001:00000bac       ??_C@_0BE@IPJGIGMK@thread?5list?5follows?$AA@ 00400f0c     dmserv.obj
 0001:00000bc0       ??_C@_06FJHNOCKE@thread?$AA@ 00400f20     dmserv.obj
 0001:00000bc8       ??_C@_09BOIBMEBJ@exception?$AA@ 00400f28     dmserv.obj
 0001:00000bd4       ??_C@_0M@DOBDBOIP@?$CFs?$DN0x?$CF04x?$AN?6?$AA@ 00400f34     dmserv.obj
 0001:00000be0       ??_C@_0M@PLODPDIO@?$CFs?$DN0x?$CF08x?$AN?6?$AA@ 00400f40     dmserv.obj
 0001:00000bec       ??_C@_02GDNLOIIJ@fp?$AA@   00400f4c     dmserv.obj
 0001:00000bf0       ??_C@_04PLMLMMEO@full?$AA@ 00400f50     dmserv.obj
 0001:00000bf8       ??_C@_03JBIPMCLC@int?$AA@  00400f58     dmserv.obj
 0001:00000bfc       ??_C@_07MMBOFDEG@control?$AA@ 00400f5c     dmserv.obj
 0001:00000c04       ??_C@_03MDPCKCMI@ext?$AA@  00400f64     dmserv.obj
 0001:00000c08       ??_C@_0BG@FGCHAFAF@name?$DN?$CC?$CFs?$CC?5type?$DN0x?$CF08x?$AA@ 00400f68     dmserv.obj
 0001:00000c20       ??_C@_0EC@HDCCDNDL@type?$DN0x?$CF08x?5vallo?$DN0x?$CF08x?5valhi?$DN0@ 00400f80     dmserv.obj
 0001:00000c64       ??_C@_0BF@ILBKCDME@counter?5data?5follows?$AA@ 00400fc4     dmserv.obj
 0001:00000c7c       ??_C@_04GPMDFGEJ@type?$AA@ 00400fdc     dmserv.obj
 0001:00000c84       ??_C@_04IAGNFIBA@size?$AA@ 00400fe4     dmserv.obj
 0001:00000c8c       ??_C@_07EMGJIMLB@execute?$AA@ 00400fec     dmserv.obj
 0001:00000c94       ??_C@_05NGFEDHGN@write?$AA@ 00400ff4     dmserv.obj
 0001:00000c9c       ??_C@_04POLDLDMI@read?$AA@ 00400ffc     dmserv.obj
 0001:00000ca4       ??_C@_05MEHLAELG@clear?$AA@ 00401004     dmserv.obj
 0001:00000cac       ??_C@_08GJHHGJFP@clearall?$AA@ 0040100c     dmserv.obj
 0001:00000cb8       ??_C@_0BG@NJCKFLII@execution?5not?5pending?$AA@ 00401018     dmserv.obj
 0001:00000cd0       ??_C@_05FAGFPHJG@start?$AA@ 00401030     dmserv.obj
 0001:00000cd8       ??_C@_03CGLHMDPP@now?$AA@  00401038     dmserv.obj
 0001:00000cdc       ??_C@_07KMJBNFCM@type?$DN?$CFd?$AA@ 0040103c     dmserv.obj
 0001:00000ce4       ??_C@_0BA@OKMLEEBI@setvalue?5failed?$AA@ 00401044     dmserv.obj
 0001:00000cf4       ??_C@_05MFEJDJP@value?$AA@ 00401054     dmserv.obj
 0001:00000cfc       ??_C@_05FKHKFDID@index?$AA@ 0040105c     dmserv.obj
 0001:00000d04       ??_C@_0BI@PIHPAMOP@debugstr?5thread?$DN?$CFd?5stop?$AA@ 00401064     dmserv.obj
 0001:00000d1c       ??_C@_0BN@NOBFDBFB@assert?5prompt?5thread?$DN?$CFd?5stop?$AA@ 0040107c     dmserv.obj
 0001:00000d3c       ??_C@_07IEOHBIGJ@stopped?$AA@ 0040109c     dmserv.obj
 0001:00000d44       ??_C@_0CG@NJBHOOCD@suspend?$DN?$CFd?5priority?$DN?$CFd?5tlsbase?$DN0@ 004010a4     dmserv.obj
 0001:00000d6c       ??_C@_0BE@OGMOMOMA@thread?5info?5follows?$AA@ 004010cc     dmserv.obj
 0001:00000d80       ??_C@_0P@HGGDCDFM@lasterr?$DN0x?$CF08x?$AA@ 004010e0     dmserv.obj
 0001:00000d90       ??_C@_0BB@FJFCHJID@xtl?5info?5follows?$AA@ 004010f0     dmserv.obj
 0001:00000da4       ??_C@_0BH@GNNNFKOA@no?5long?5name?5available?$AA@ 00401104     dmserv.obj
 0001:00000dbc       ??_C@_0BB@HDAEGOHB@timestamp?$DN0x?$CF08x?$AA@ 0040111c     dmserv.obj
 0001:00000dd0       ??_C@_0BA@NDDPPEOF@checksum?$DN0x?$CF08x?$AA@ 00401130     dmserv.obj
 0001:00000de0       ??_C@_05DFCJAACA@name?$DN?$AA@ 00401140     dmserv.obj
 0001:00000de8       ??_C@_07PANPENDC@running?$AA@ 00401148     dmserv.obj
 0001:00000df0       ??_C@_0L@CNHMCLA@no?5command?$AA@ 00401150     dmserv.obj
 0001:00000dfc       ??_C@_0L@KKPFIJOL@disconnect?$AA@ 0040115c     dmserv.obj
 0001:00000e08       ??_C@_07KAIBNCHO@connect?$AA@ 00401168     dmserv.obj
 0001:00000e10       ??_C@_0BD@EFOMABGG@high?$DN0x?$CFx?5low?$DN0x?$CFx?$AA@ 00401170     dmserv.obj
 0001:00000e24       ??_C@_0M@LEMHMAEF@addr?$DN0x?$CF08x?$AA@ 00401184     dmserv.obj
 0001:00000e30       ??_C@_03LMPCJCAN@PDT?$AA@  00401190     dmserv.obj
 0001:00000e34       ??_C@_03KFJLCHPI@PST?$AA@  00401194     dmserv.obj
 0001:00000e38       ??_C@_02IGJGHHBN@tz?$AA@   00401198     dmserv.obj
 0001:00000e3c       ??_C@_07OABACEGD@clocklo?$AA@ 0040119c     dmserv.obj
 0001:00000e44       ??_C@_07LBEDCLDJ@clockhi?$AA@ 004011a4     dmserv.obj
 0001:00000e4c       ??_C@_07JFMHDDB@nodebug?$AA@ 004011ac     dmserv.obj
 0001:00000e54       ??_C@_04HGJDANIP@warm?$AA@ 004011b4     dmserv.obj
 0001:00000e5c       ??_C@_07EMONB@200?9?5OK?$AA@ 004011bc     dmserv.obj
 0001:00000e64       ??_C@_05GFCDIDHO@debug?$AA@ 004011c4     dmserv.obj
 0001:00000e6c       ??_C@_0O@LNFKOLDO@missing?5title?$AA@ 004011cc     dmserv.obj
 0001:00000e7c       ??_C@_0P@MKJMMOJE@E?3?2xboxcap?4dat?$AA@ 004011dc     dmserv.obj
 0001:00000e8c       ??_C@_0BE@BLPHLHLO@error?5status?50x?$CF08x?$AA@ 004011ec     dmserv.obj
 0001:00000ea0       ??_C@_0M@JDHFKJFN@flashing?4?4?4?$AA@ 00401200     dmserv.obj
 0001:00000eac       ??_C@_0CC@FPNHPNJI@bad?5data?5detected?5in?5kernel?5imag@ 0040120c     dmserv.obj
 0001:00000ed0       ??_C@_0BF@DMJAHBCD@Invalid?5parameter?$CIs?$CJ?$AA@ 00401230     dmserv.obj
 0001:00000ee8       ??_C@_0BK@MPIPGFEN@Invalid?5kernel?5image?5size?$AA@ 00401248     dmserv.obj
 0001:00000f04       ??_C@_0BC@BAKIAKOF@Not?5enough?5memory?$AA@ 00401264     dmserv.obj
 0001:00000f18       ??_C@_0BG@FNAFBLLO@ignoreversionchecking?$AA@ 00401278     dmserv.obj
 0001:00000f30       ??_C@_03OOINPMFE@crc?$AA@  00401290     dmserv.obj
 0001:00000f38       ??_C@_0IE@LIEGEDAP@freetocallerlo?$DN0x?$CF08x?5freetocall@ 00401298     dmserv.obj
 0001:00000fbc       ??_C@_0BD@CCPGFPGB@unknown?5error?5?$CI?$CFd?$CJ?$AA@ 0040131c     dmserv.obj
 0001:00000fd0       ??_C@_0EO@MFLGHHPK@pitch?$DN0x?$CF08x?5width?$DN0x?$CF08x?5height@ 00401330     dmserv.obj
 0001:00001020       ??_C@_0P@PECENKIC@can?8t?5lock?5GPU?$AA@ 00401380     dmserv.obj
 0001:00001030       ??_C@_0BO@DIIEIMPK@Unexpected?5framebuffer?5format?$AA@ 00401390     dmserv.obj
 0001:00001050       ??_C@_0BJ@GCPPEPAA@can?8t?5find?5screen?5buffer?$AA@ 004013b0     dmserv.obj
 0001:00001070       ??_C@_0GG@HFKKGHCO@The?5Application?5is?5using?5an?5unsu@ 004013d0     dmserv.obj
 0001:000010d8       ??_C@_0FH@IANNLFKM@Debugger?5doesn?8t?5support?5an?5Xbox@ 00401438     dmserv.obj
 0001:00001130       ??_C@_0CJ@HDHPJAND@Debugger?5wasn?8t?5able?5to?5allocate@ 00401490     dmserv.obj
 0001:0000115c       ??_C@_0CG@FCCPEANE@D3D?5snapshot?5client?5returned?5err@ 004014bc     dmserv.obj
 0001:00001184       ??_C@_0CP@HODGJOPL@Opcode?5timeout?3?5?5Failed?5to?5recei@ 004014e4     dmserv.obj
 0001:000011b4       ??_C@_0CM@LLENMENO@D3D?5snapshot?5client?5in?5invalid?5s@ 00401514     dmserv.obj
 0001:000011e0       ??_C@_06HHHKAAEJ@marker?$AA@ 00401540     dmserv.obj
 0001:000011e8       ??_C@_05GECEPKB@flags?$AA@ 00401548     dmserv.obj
 0001:000011f0       ??_C@_0BE@MIMOEGGC@Missing?5Y?5parameter?$AA@ 00401550     dmserv.obj
 0001:00001204       ??_C@_01EANLCPLP@y?$AA@    00401564     dmserv.obj
 0001:00001208       ??_C@_0BE@FDGLAKAN@Missing?5X?5parameter?$AA@ 00401568     dmserv.obj
 0001:0000121c       ??_C@_01FJMABOPO@x?$AA@    0040157c     dmserv.obj
 0001:00001220       ??_C@_0DF@KFGHHCKF@Opcode?5timeout?3?5?5Failed?5to?5recei@ 00401580     dmserv.obj
 0001:00001258       ??_C@_0BH@NHEHMDCE@Missing?5Last?5parameter?$AA@ 004015b8     dmserv.obj
 0001:00001270       ??_C@_04PLGBGIDD@last?$AA@ 004015d0     dmserv.obj
 0001:00001278       ??_C@_05NIGAKFML@first?$AA@ 004015d8     dmserv.obj
 0001:00001280       ??_C@_0CM@OGOKMMGI@box?5not?5locked?$DL?5file?5encryption?5@ 004015e0     dmserv.obj
 0001:000012ac       ??_C@_07NNLIEMBO@encrypt?$AA@ 0040160c     dmserv.obj
 0001:000012b4       ??_C@_0BD@FMCFODNL@missing?5parameters?$AA@ 00401614     dmserv.obj
 0001:000012c8       ??_C@_06BNCCALCL@unlock?$AA@ 00401628     dmserv.obj
 0001:000012d0       ??_C@_0BB@LNNDIIOH@boxid?$DN0q?$CF08x?$CF08x?$AA@ 00401630     dmserv.obj
 0001:000012e4       ??_C@_0BB@FCLDBLDL@missing?5response?$AA@ 00401644     dmserv.obj
 0001:000012f8       ??_C@_05JEBDMKHG@admin?$AA@ 00401658     dmserv.obj
 0001:00001300       ??_C@_04MPLPBDID@resp?$AA@ 00401660     dmserv.obj
 0001:00001308       ??_C@_06NKIEGJEO@passwd?$AA@ 00401668     dmserv.obj
 0001:00001310       ??_C@_0P@HNKJKDFK@missing?5passwd?$AA@ 00401670     dmserv.obj
 0001:00001320       ??_C@_02FIDLOBHM@me?$AA@   00401680     dmserv.obj
 0001:00001328       ??_C@_0IE@MFDLHFEM@MmHighestPhysicalPage?$DN0x?$CFx?5Retai@ 00401688     dmserv.obj
 0001:000013b0       ??_C@_0HE@IBADHDCI@AddressSpaceLock?$DN0x?$CFx?5VadRoot?$DN0x@ 00401710     dmserv.obj
 0001:00001424       ??_C@_0P@PPFCKJAD@?2Device?2Cdrom0?$AA@ 00401784     dmserv.obj
 0001:00001434       ??_C@_05PIBOEKAB@block?$AA@ 00401794     dmserv.obj
 0001:0000143c       ??_C@_0BK@OIKOFOJO@205?9?5connection?5dedicated?$AA@ 0040179c     dmserv.obj
 0001:00001458       ??_C@_0DE@ICNBLPHE@dm?3?5rededicating?5a?5connection?5on@ 004017b8     dmserv.obj
 0001:0000148c       ??_C@_0BA@NCMGMANN@missing?5handler?$AA@ 004017ec     dmserv.obj
 0001:0000149c       ??_C@_07MILLDJGK@handler?$AA@ 004017fc     dmserv.obj
 0001:000014a4       ??_C@_06FJKEMHGD@global?$AA@ 00401804     dmserv.obj
 0001:000014ac       ??_C@_07LKOIKIBH@?5manage?$AA@ 0040180c     dmsecure.obj
 0001:000014b4       ??_C@_07HFKCMFAL@?5config?$AA@ 00401814     dmsecure.obj
 0001:000014bc       ??_C@_08MNMEBKCC@?5control?$AA@ 0040181c     dmsecure.obj
 0001:000014c8       ??_C@_06DFEHHACM@?5write?$AA@ 00401828     dmsecure.obj
 0001:000014d0       ??_C@_05IOPPOAEA@?5read?$AA@ 00401830     dmsecure.obj
 0001:000014d8       ??_C@_06LLNAMKFG@manage?$AA@ 00401838     dmsecure.obj
 0001:000014e0       ??_C@_06HEJKKHEK@config?$AA@ 00401840     dmsecure.obj
 0001:000014e8       ??_C@_0M@HJKICNFN@name?$DN?$CC?$CFs?$CC?$CFs?$AA@ 00401848     dmsecure.obj
 0001:000014f4       ??_C@_0BD@CAJKCLKJ@?5passwd?$DN0q?$CF08x?$CF08x?$AA@ 00401854     dmsecure.obj
 0001:00001508       ??_C@_05GFKJMHJM@user?5?$AA@ 00401868     dmsecure.obj
 0001:00001510       ??_C@_0BK@PIDLIHJG@adminpw?5passwd?$DN0q?$CF08x?$CF08x?$AA@ 00401870     dmsecure.obj
 0001:0000152c       ??_C@_0BM@BOCFAMBM@lockmode?5boxid?$DN0q?$CF08x?$CF08x?$CFs?$AA@ 0040188c     dmsecure.obj
 0001:00001548       ??_C@_08NMGCAFHK@?5encrypt?$AA@ 004018a8     dmsecure.obj
 0001:00001554       ??_C@_06LEMKAMD@remove?$AA@ 004018b4     dmsecure.obj
 0001:0000155c       ??_C@_07JPJEMOCA@pending?$AA@ 004018bc     dmnotify.obj
 0001:00001564       ??_C@_09MMCGMFEO@rebooting?$AA@ 004018c4     dmnotify.obj
 0001:00001570       ??_C@_07ELEPLNCO@started?$AA@ 004018d0     dmnotify.obj
 0001:00001578       ??_C@_0CE@BHPFBJKB@notifyat?5addr?$DN?$CFd?4?$CFd?4?$CFd?4?$CFd?5port?$DN?$CF@ 004018d8     dmnotify.obj
 0001:0000159c       ??_C@_06IGDAMEDP@?5debug?$AA@ 004018fc     dmnotify.obj
 0001:000015a4       ??_C@_09GIJGGOJL@?$CFsstring?$DN?$AA@ 00401904     dmnotify.obj
 0001:000015b0       ??_C@_03HGJFPLGI@lf?5?$AA@ 00401910     dmnotify.obj
 0001:000015b4       ??_C@_05OLGBELIM@crlf?5?$AA@ 00401914     dmnotify.obj
 0001:000015bc       ??_C@_03DFNJOAJC@cr?5?$AA@ 0040191c     dmnotify.obj
 0001:000015c0       ??_C@_0BA@DJNEDPCP@?$CFs?5?$CFsthread?$DN?$CFd?5?$AA@ 00401920     dmnotify.obj
 0001:000015d0       ??_C@_05GNOJMMJL@stop?5?$AA@ 00401930     dmnotify.obj
 0001:000015d8       ??_C@_06GMEIIFFN@assert?$AA@ 00401938     dmnotify.obj
 0001:000015e0       ??_C@_0EE@IMKIMBDG@name?$DN?$CC?$CFs?$CC?5base?$DN0x?$CF08x?5size?$DN0x?$CF08@ 00401940     dmnotify.obj
 0001:00001624       ??_C@_04FJJOAIFM@?5tls?$AA@ 00401984     dmnotify.obj
 0001:0000162c       ??_C@_04FEOCPDJ@?5xbe?$AA@ 0040198c     dmnotify.obj
 0001:00001634       ??_C@_0DE@EMJDKFME@name?$DN?$CC?$CFs?$CC?5base?$DN0x?$CF08x?5size?$DN0x?$CF08@ 00401994     dmnotify.obj
 0001:00001668       ??_C@_08KFKLDJEN@?5noncont?$AA@ 004019c8     dmnotify.obj
 0001:00001674       ??_C@_06DLHDOCIK@?5first?$AA@ 004019d4     dmnotify.obj
 0001:0000167c       ??_C@_0L@BHPAIFBB@?5?$CFs?$DN0x?$CF08x?$AA@ 004019dc     dmnotify.obj
 0001:00001688       ??_C@_0CP@DDBJNEDM@exception?5code?$DN0x?$CF08x?5thread?$DN?$CFd?5@ 004019e8     dmnotify.obj
 0001:000016b8       ??_C@_0CG@MPPJHHBL@data?5?$CFs?$DN0x?$CF08x?5addr?$DN0x?$CF08x?5threa@ 00401a18     dmnotify.obj
 0001:000016e0       ??_C@_0P@KPFBPGJI@rip?5thread?$DN?$CFlu?$AA@ 00401a40     dmnotify.obj
 0001:000016f0       ??_C@_0BP@GMDKCEDB@rip?$CFs?5thread?$DN?$CFlu?5string?$DN?$CF?9?$CK?4?$CKs?$AA@ 00401a50     dmnotify.obj
 0001:00001710       ??_C@_05HPAKADFF@?5stop?$AA@ 00401a70     dmnotify.obj
 0001:00001718       ??_C@_09GMCIMGBM@sectload?5?$AA@ 00401a78     dmnotify.obj
 0001:00001724       ??_C@_0M@GDEPCNIN@sectunload?5?$AA@ 00401a84     dmnotify.obj
 0001:00001730       ??_C@_0BE@CCMPAOFI@terminate?5thread?$DN?$CFd?$AA@ 00401a90     dmnotify.obj
 0001:00001744       ??_C@_0BM@MKBJBGDL@break?5addr?$DN0x?$CF08x?5thread?$DN?$CFd?$AA@ 00401aa4     dmnotify.obj
 0001:00001760       ??_C@_0N@BDEEMHFG@execution?5?$CFs?$AA@ 00401ac0     dmnotify.obj
 0001:00001770       ??_C@_0CB@DDNFLKOF@singlestep?5addr?$DN0x?$CF08x?5thread?$DN?$CFd@ 00401ad0     dmnotify.obj
 0001:00001794       ??_C@_08PPHMKPMG@modload?5?$AA@ 00401af4     dmnotify.obj
 0001:000017a0       ??_C@_0BO@EDBLMNGO@create?5thread?$DN?$CFd?5start?$DN0x?$CF08x?$AA@ 00401b00     dmnotify.obj
 0001:000017c0       ??_C@_04MLLLIHIP@null?$AA@ 00401b20     dmnotify.obj
 0001:000017c8       ??_C@_0BI@DHHIOCDN@assert?5prompt?5thread?$DN?$CFd?$AA@ 00401b28     dmnotify.obj
 0001:000017e0       ??_C@_0CA@OGCHDGFJ@205?9?5now?5a?5notification?5channel?$AA@ 00401b40     dmnotify.obj
 0001:00001800       ??_C@_04PIONEEJD@drop?$AA@ 00401b60     dmnotify.obj
 0001:00001808       ??_C@_04LPGMAPLE@port?$AA@ 00401b68     dmnotify.obj
 0001:00001810       ??_C@_05CJBACGMB@hello?$AA@ 00401b70     dmnotify.obj
 0001:00001818       ??_C@_0CN@GFIOFMHL@xbdm?5callback?3?5timed?5out?5waiting@ 00401b78     dmnotify.obj
 0001:00001848       ??_C@_07KKMMDFCO@?4bistro?$AA@ 00401ba8     dmmodule.obj
 0001:00001850       ??_C@_08EJOALOPG@xbdm?4dll?$AA@ 00401bb0     dmmodule.obj
 0001:0000185c       ??_C@_04PONNOKHC@xbdm?$AA@ 00401bbc     dmmodule.obj
 0001:00001874       _oszCounterDir             00401bd4     dmcount.obj
 0001:00001880       ??_C@_0O@FMKPGBFN@?$CF?5GPU?5Backend?$AA@ 00401be0     dmcount.obj
 0001:00001890       ??_C@_0P@KLLEAMGN@?$CF?5GPU?5Frontend?$AA@ 00401bf0     dmcount.obj
 0001:000018a0       ??_C@_05HFCOACPI@?$CF?5GPU?$AA@ 00401c00     dmcount.obj
 0001:000018a8       ??_C@_08CBLIIHED@VM?5Pages?$AA@ 00401c08     dmcount.obj
 0001:000018b4       ??_C@_0M@NMOAHNAN@Stack?5Pages?$AA@ 00401c14     dmcount.obj
 0001:000018c0       ??_C@_0L@EDCKLEJJ@Pool?5Pages?$AA@ 00401c20     dmcount.obj
 0001:000018cc       ??_C@_0M@KHBCMBOA@Image?5Pages?$AA@ 00401c2c     dmcount.obj
 0001:000018d8       ??_C@_0M@JMHDKEKK@Cache?5Pages?$AA@ 00401c38     dmcount.obj
 0001:000018e4       ??_C@_0L@FNFICBPM@Free?5Pages?$AA@ 00401c44     dmcount.obj
 0001:000018f0       ??_C@_0BB@IKIBEMCK@?$CF?5CPU?3Interrupts?$AA@ 00401c50     dmcount.obj
 0001:00001904       ??_C@_09KHHLDFHI@?$CF?5CPU?3DPC?$AA@ 00401c64     dmcount.obj
 0001:00001910       ??_C@_0M@HLPPPNPI@?$CF?5CPU?3total?$AA@ 00401c70     dmcount.obj
 0001:0000191c       ??_C@_06CELCJONF@Frames?$AA@ 00401c7c     dmcount.obj
 0001:00001924       ??_C@_0CM@FEIBHMDD@Failed?5to?5create?5counter?5object?5@ 00401c84     dmcount.obj
 0001:00001950       _EDRIVE_OBNAME             00401cb0     dmfile.obj
 0001:00001974       _SDRIVE_OBNAME             00401cd4     dmfile.obj
 0001:00001998       _VDRIVE_OBNAME             00401cf8     dmfile.obj
 0001:000019bc       _CDROM_OBNAME              00401d1c     dmfile.obj
 0001:000019cc       _CDDEVKIT_OBNAME           00401d2c     dmfile.obj
 0001:000019e4       _ILLEGAL_OBNAME            00401d44     dmfile.obj
 0001:000019f0       _SYMLINK_OBNAME            00401d50     dmfile.obj
 0001:000019fc       ??_C@_0BM@CPPIHIHH@DmFreePool?5called?5for?5?$CF08x?6?$AA@ 00401d5c     dmpool.obj
 0001:00001a38       _CrcTable32                00401d98     crc.obj
 0001:00001e38       ??_C@_1BC@HOJAFCFJ@?$BP?$AH?$BP?$AI?$BP?$AL?54?5?$LA?B4?B?$LA?Z?$IM?$AA?$AA@ 00402198     flash.obj
 0001:00001e4c       ??_C@_19KPCMJDGA@?$BP?$BD?5?b?B?$KE?$KN?$KE?$AA?$AA@ 004021ac     flash.obj
 0001:00001e58       ??_C@_17FAOPPJO@?$AB?U?$AE?U?$KN?U?$AA?$AA@ 004021b8     flash.obj
 0001:00001e60       ??_C@_13MJABDJIC@?$LPS?$AA?$AA@ 004021c0     flash.obj
 0001:00001e64       ??_C@_0CI@HIFKKNMK@FLASH?3?5blank?5check?5failed?5?$CIretri@ 004021c4     flash.obj
 0001:00001e8c       ??_C@_0CJ@DHMAKEPO@FLASH?3?5verification?5failed?5?$CIretr@ 004021ec     flash.obj
 0001:00001eb8       ??_C@_0CD@NHLIIEIK@FLASH?3?5interrupts?5are?5now?5enable@ 00402218     flash.obj
 0001:00001edc       ??_C@_0BI@LLDPCHAL@Done?0?5new?5image?5flashed?$AA@ 0040223c     flash.obj
 0001:00001ef4       ??_C@_0BA@EHHAGELF@FLASH?3?5done?4?4?4?6?$AA@ 00402254     flash.obj
 0001:00001f04       ??_C@_0CP@OGCEHBEO@Failed?5to?5program?5kernel?5image?5?$CI@ 00402264     flash.obj
 0001:00001f34       ??_C@_0BH@KPKCLFMP@FLASH?3?5programming?4?4?4?6?$AA@ 00402294     flash.obj
 0001:00001f4c       ??_C@_0BL@DDHHHOM@Failed?5to?5erase?5flash?5chip?$AA@ 004022ac     flash.obj
 0001:00001f68       ??_C@_0CG@KPMHIEIC@FLASH?3?5erasing?5and?5blank?5checkin@ 004022c8     flash.obj
 0001:00001f90       ??_C@_0CI@OBKLPJLK@Mismatch?5ROM?5version?5?$CIrom?$DN?$CFx?0?5im@ 004022f0     flash.obj
 0001:00001fb8       ??_C@_0BD@BGOMCCDB@Invalid?5image?5size?$AA@ 00402318     flash.obj
 0001:00001fcc       ??_C@_0BI@JEBPBFAP@Unknown?5flash?5device?5id?$AA@ 0040232c     flash.obj
 0001:00001fe4       ??_C@_0CE@LOGPJCEC@FLASH?3?5interrupts?5are?5now?5disabl@ 00402344     flash.obj
 0001:00002008       ??_C@_0BI@KOCJIMHK@unable?5to?5map?5i?1o?5space?$AA@ 00402368     flash.obj
 0001:00002020       ??_C@_0BB@PBJLGCAA@File?5write?5error?$AA@ 00402380     sysfileupd.obj
 0001:00002034       ??_C@_0BL@KCJFOIJC@Replace?5file?5failed?5?$CI0x?$CFX?$CJ?$AA@ 00402394     sysfileupd.obj
 0001:00002050       ??_C@_0BF@CAPFPECN@Unexpected?5data?5size?$AA@ 004023b0     sysfileupd.obj
 0001:00002068       ??_C@_0M@GNAOKGLG@Invalid?5CRC?$AA@ 004023c8     sysfileupd.obj
 0001:00002074       ??_C@_0BC@JFFNKLNA@Invalid?5file?5name?$AA@ 004023d4     sysfileupd.obj
 0001:00002088       ??_C@_09BFDAEIFK@Disk?5full?$AA@ 004023e8     sysfileupd.obj
 0001:00002094       ??_C@_0O@IHGFJCHC@?2temp?$CF04x?4tmp?$AA@ 004023f4     sysfileupd.obj
 0001:000020a4       ??_C@_0BN@OEMOLBLB@missing?5or?5invalid?5file?5name?$AA@ 00402404     sysfileupd.obj
 0001:000020c4       ??_7CXbdmServer@CXnNic@@6B@ 00402424     xnetm:xnet.obj
 0001:000020fc       ??_C@_06IDFKHCBC@?2?$DP?$DP?2D?3?$AA@ 0040245c     dmxapi:launch.obj
 0001:00002138       ___lookuptable             00402498     libcntpr:output.obj
 0001:00002194       ___nullstring              004024f4     libcntpr:output.obj
 0001:0000219c       ___wnullstring             004024fc     libcntpr:output.obj
 0001:00002200       _MulDiv@12                 00402560 f   muldiv.obj
 0001:00002320       _DmpThreadStartup@8        00402680 f   thread.obj
 0001:00002340       _CallOnStack@12            004026a0 f   thread.obj
 0001:00002370       _SetDreg@20                004026d0 f   dbregs.obj
 0001:000023e8       @DwExchangeDr6@4           00402748 f   dbregs.obj
 0001:000023f0       _SetupFuncCall@0           00402750 f   funccall.obj
 0001:00002450       _QueueDfn@4                004027b0 f   defer.obj
 0001:00002468       _ProcessDfns@0             004027c8 f   defer.obj
 0001:000024a0       _CallDxtEntry@8            00402800 f   dxtstart.obj
 0001:000024b8       _FInitThreadDebugData@4    00402818 f   dminit.obj
 0001:0000252a       _DoIniLine@4               0040288a f   dminit.obj
 0001:000025e4       _LoadIniFile@0             00402944 f   dminit.obj
 0001:000026cd       _LoadPlugIns@0             00402a2d f   dminit.obj
 0001:0000278c       _WriteIniData@12           00402aec f   dminit.obj
 0001:00002843       _WriteIniSzNoCRLF@8        00402ba3 f   dminit.obj
 0001:00002864       _WriteIniSz@8              00402bc4 f   dminit.obj
 0001:00002884       _WriteIniFile@0            00402be4 f   dminit.obj
 0001:000029ca       _DisableAPIC@4             00402d2a f   dminit.obj
 0001:000029e3       _PsGetCurrentThreadId@0    00402d43 f   dminit.obj
 0001:000029f0       _CreateThreadNotify@12     00402d50 f   dminit.obj
 0001:00002aca       _DmEntryPoint@12           00402e2a f   dminit.obj
 0001:00002d45       _BindUDP@4                 004030a5 f   dmserv.obj
 0001:00002da4       _PingAllXboxes@0           00403104 f   dmserv.obj
 0001:00002ef4       _InitServ@0                00403254 f   dmserv.obj
 0001:00002f2f       _StopServ@0                0040328f f   dmserv.obj
 0001:00002f9d       _SgnCompareRgch@12         004032fd f   dmserv.obj
 0001:00003001       _FEqualRgch@12             00403361 f   dmserv.obj
 0001:0000301a       _DwHexFromSz@8             0040337a f   dmserv.obj
 0001:00003075       _DwFromSz@8                004033d5 f   dmserv.obj
 0001:000030e1       _CloseConn@4               00403441 f   dmserv.obj
 0001:00003124       _InitDmcc@4                00403484 f   dmserv.obj
 0001:00003159       _PrintSockLine@8           004034b9 f   dmserv.obj
 0001:000031ee       _FIsSpace@4                0040354e f i dmserv.obj
 0001:00003208       _PchGetParam@12            00403568 f   dmserv.obj
 0001:000032d9       _CchOfWord@4               00403639 f   dmserv.obj
 0001:000032fe       _GetParam@12               0040365e f   dmserv.obj
 0001:00003373       _FGetSzParam@16            004036d3 f   dmserv.obj
 0001:0000339a       _FGetDwParam@12            004036fa f   dmserv.obj
 0001:000033e1       _FGetQwordParam@12         00403741 f   dmserv.obj
 0001:000034be       _FGetNamedDwParam@16       0040381e f   dmserv.obj
 0001:000034f1       _UlAddrFromSz@4            00403851 f   dmserv.obj
 0001:00003554       _SzStdResponse@4           004038b4 f   dmserv.obj
 0001:00003710       _HrFromStatus@8            00403a70 f   dmserv.obj
 0001:000037a6       _DmplOfConnection@4        00403b06 f   dmserv.obj
 0001:000037cf       _SendHrSzResp@16           00403b2f f   dmserv.obj
 0001:00003875       _HrHandleBuiltinCommand@24 00403bd5 f   dmserv.obj
 0001:00003944       _DoSendReceive@8           00403ca4 f   dmserv.obj
 0001:00003bd0       _PechFindHandler@8         00403f30 f   dmserv.obj
 0001:00003c05       _HandleCommand@8           00403f65 f   dmserv.obj
 0001:00003e0b       _AnswerName@4              0040416b f   dmserv.obj
 0001:00003f17       _HandleSocketRead@4        00404277 f   dmserv.obj
 0001:00004045       _DedicatedServThread@4     004043a5 f   dmserv.obj
 0001:00004130       _ServerThread@4            00404490 f   dmserv.obj
 0001:000045a4       _FStartDebugService@0      00404904 f   dmserv.obj
 0001:000045c6       _DmSetXboxName@4           00404926 f   dmserv.obj
 0001:00004600       _DmGetXboxName@8           00404960 f   dmserv.obj
 0001:0000465b       _DmRegisterCommandProcessorEx@12 004049bb f   dmserv.obj
 0001:00004764       _DmThreadUserData@8        00404ac4 f   dmserv.obj
 0001:000047d7       _HrEndConversation@16      00404b37 f   dmserv.obj
 0001:00004818       _HrSetDbgName@16           00404b78 f   dmserv.obj
 0001:0000489e       _HrToggleGPUCounters@16    00404bfe f   dmserv.obj
 0001:000048dc       _HrToggleKDState@16        00404c3c f   dmserv.obj
 0001:00004994       _HrSetupNotifyAt@16        00404cf4 f   dmserv.obj
 0001:000049e7       _HrSetupNotify@16          00404d47 f   dmserv.obj
 0001:00004a3b       _HrDoStopon@20             00404d9b f   dmserv.obj
 0001:00004ac2       _HrStopon@16               00404e22 f   dmserv.obj
 0001:00004adc       _HrNostopon@16             00404e3c f   dmserv.obj
 0001:00004af6       _HrGo@16                   00404e56 f   dmserv.obj
 0001:00004b23       _HrStop@16                 00404e83 f   dmserv.obj
 0001:00004b50       _FTitleExists@16           00404eb0 f   dmserv.obj
 0001:00004cae       _HrReceiveFileData@12      0040500e f   dmserv.obj
 0001:00004da9       _HrReceiveFile@16          00405109 f   dmserv.obj
 0001:00004ed5       _HrSendFileData@12         00405235 f   dmserv.obj
 0001:00004f71       _HrSendFile@16             004052d1 f   dmserv.obj
 0001:00005072       _GetFileAttrSz@20          004053d2 f   dmserv.obj
 0001:000050d0       _HrReportFileAttributes@12 00405430 f   dmserv.obj
 0001:00005108       _HrGetFileAttributes@16    00405468 f   dmserv.obj
 0001:000051cd       _HrSetFileAttributes@16    0040552d f   dmserv.obj
 0001:00005341       _HrRenameFile@16           004056a1 f   dmserv.obj
 0001:00005462       _HrDeleteFile@16           004057c2 f   dmserv.obj
 0001:00005596       _HrReportDirList@12        004058f6 f   dmserv.obj
 0001:0000567f       _HrGetDirList@16           004059df f   dmserv.obj
 0001:00005730       _HrMkdir@16                00405a90 f   dmserv.obj
 0001:000057c0       _HrFormatFAT@16            00405b20 f   dmserv.obj
 0001:00005862       _DmSetTitle@12             00405bc2 f   dmserv.obj
 0001:00005925       _HrSetTitle@16             00405c85 f   dmserv.obj
 0001:000059a1       _HrSetDefaultTitle@16      00405d01 f   dmserv.obj
 0001:00005c3c       _HrReportMemory@12         00405f9c f   dmserv.obj
 0001:00005d7f       _HrGetMemory@16            004060df f   dmserv.obj
 0001:00005dfb       _HrSetMemory@16            0040615b f   dmserv.obj
 0001:00005f36       _HrReportThreads@12        00406296 f   dmserv.obj
 0001:00005fad       _HrListThreads@16          0040630d f   dmserv.obj
 0001:0000602f       _HrHaltThread@16           0040638f f   dmserv.obj
 0001:00006056       _HrContinueThread@16       004063b6 f   dmserv.obj
 0001:00006094       _HrSuspendThread@16        004063f4 f   dmserv.obj
 0001:000060c2       _HrResumeThread@16         00406422 f   dmserv.obj
 0001:000060f0       _HrFunctionCall@16         00406450 f   dmserv.obj
 0001:0000611e       _PcregNext@4               0040647e f   dmserv.obj
 0001:00006216       _HrDoExtContext@12         00406576 f   dmserv.obj
 0001:000062f8       _HrGetExtContext@16        00406658 f   dmserv.obj
 0001:000063b4       _HrReportContext@12        00406714 f   dmserv.obj
 0001:00006446       _HrGetContext@16           004067a6 f   dmserv.obj
 0001:0000655e       _HrSetContext@16           004068be f   dmserv.obj
 0001:000066ef       _FillSzFromWz@16           00406a4f f   dmserv.obj
 0001:00006745       _HrReportCounters@12       00406aa5 f   dmserv.obj
 0001:000067ae       _HrListCounters@16         00406b0e f   dmserv.obj
 0001:000067d1       _HrReportCounterData@12    00406b31 f   dmserv.obj
 0001:00006813       _HrQueryPerformanceCounter@16 00406b73 f   dmserv.obj
 0001:000068cf       _HrReportModules@12        00406c2f f   dmserv.obj
 0001:0000692d       _HrListModules@16          00406c8d f   dmserv.obj
 0001:00006950       _HrReportModuleSections@12 00406cb0 f   dmserv.obj
 0001:000069b0       _HrListModuleSections@16   00406d10 f   dmserv.obj
 0001:00006a36       _HrDoBreak@16              00406d96 f   dmserv.obj
 0001:00006b89       _HrIsBreak@16              00406ee9 f   dmserv.obj
 0001:00006bd9       _HrSetConfig@16            00406f39 f   dmserv.obj
 0001:00006c44       _HrIsStopped@16            00406fa4 f   dmserv.obj
 0001:00006ccf       _HrReportThreadInfo@12     0040702f f   dmserv.obj
 0001:00006d0b       _HrThreadInfo@16           0040706b f   dmserv.obj
 0001:00006d6f       _HrReportXapiInfo@12       004070cf f   dmserv.obj
 0001:00006da3       _HrXapiInfo@16             00407103 f   dmserv.obj
 0001:00006de5       _HrDoLongName@16           00407145 f   dmserv.obj
 0001:00006e4a       _HrReportXbeInfo@12        004071aa f   dmserv.obj
 0001:00006eda       _HrXbeInfo@16              0040723a f   dmserv.obj
 0001:00006f95       _DmIsDebuggerPresent@0     004072f5 f   dmserv.obj
 0001:00006f9b       _HrConnectDebugger@16      004072fb f   dmserv.obj
 0001:0000700c       _HrSystemTime@16           0040736c f   dmserv.obj
 0001:0000704a       _HrGetAltAddr@16           004073aa f   dmserv.obj
 0001:0000708b       _HrSetSystemTime@16        004073eb f   dmserv.obj
 0001:000071a6       _HrReboot@16               00407506 f   dmserv.obj
 0001:00007235       _HrMagicReboot@16          00407595 f   dmserv.obj
 0001:0000738a       _CAPGetFileHeader@0        004076ea f   dmserv.obj
 0001:0000741b       _CAPWriteFile@4            0040777b f   dmserv.obj
 0001:0000754e       _HrCAPControl@16           004078ae f   dmserv.obj
 0001:000075de       _HrIrtSweep@16             0040793e f   dmserv.obj
 0001:000075fc       _HrReceiveKernelImage@12   0040795c f   dmserv.obj
 0001:000076e2       _HrFlashKernelImage@16     00407a42 f   dmserv.obj
 0001:000077e2       _HrGetDriveList@16         00407b42 f   dmserv.obj
 0001:00007989       _HrReportDriveFreeSpace@12 00407ce9 f   dmserv.obj
 0001:00007a42       _HrGetDriveFreeSpace@16    00407da2 f   dmserv.obj
 0001:00007ad7       _HrSendFrameData@12        00407e37 f   dmserv.obj
 0001:00007b65       _HrScreenshot@16           00407ec5 f   dmserv.obj
 0001:00007c70       _HrSendPSSnapshotData@12   00407fd0 f   dmserv.obj
 0001:00007ca2       _HrPSSnap@16               00408002 f   dmserv.obj
 0001:00007e2e       _HrSendVSSnapshotData@12   0040818e f   dmserv.obj
 0001:00007e60       _HrVSSnap@16               004081c0 f   dmserv.obj
 0001:00008117       _HrSetLockMode@16          00408477 f   dmserv.obj
 0001:000081c6       _HrSetDebugSecureMode@16   00408526 f   dmserv.obj
 0001:00008207       _HrGetBoxId@16             00408567 f   dmserv.obj
 0001:0000823c       _HrAuthenticateUser@16     0040859c f   dmserv.obj
 0001:00008353       _HrSetAdminPasswd@16       004086b3 f   dmserv.obj
 0001:0000840e       _HrGetUserPriv@16          0040876e f   dmserv.obj
 0001:000084c0       _HrSetUserPriv@16          00408820 f   dmserv.obj
 0001:00008510       _HrReportUsers@12          00408870 f   dmserv.obj
 0001:00008566       _HrListUsers@16            004088c6 f   dmserv.obj
 0001:00008599       _HrPerformDHExchange@12    004088f9 f   dmserv.obj
 0001:000086a6       _HrKeyExchange@16          00408a06 f   dmserv.obj
 0001:000086f1       _HrReportMmGlobal@12       00408a51 f   dmserv.obj
 0001:000087b4       _HrGetMmGlobal@16          00408b14 f   dmserv.obj
 0001:000087cd       _HrReturnBuffer@12         00408b2d f   dmserv.obj
 0001:000087f6       _HrGetDvdBlk@16            00408b56 f   dmserv.obj
 0001:000088c3       _FDedicateConnection@8     00408c23 f   dmserv.obj
 0001:00008978       _DmRegisterCommandProcessor@8 00408cd8 f   dmserv.obj
 0001:0000898a       _HrDedicateConnection@16   00408cea f   dmserv.obj
 0001:00008a3c       _XBCEncryptCore@8          00408d9c f   dmsecure.obj
 0001:00008aa9       _XBCHashBlock@8            00408e09 f   dmsecure.obj
 0001:00008ae1       _XBCHashData@12            00408e41 f   dmsecure.obj
 0001:00008b4a       _XBCCross@12               00408eaa f   dmsecure.obj
 0001:00008b8f       _InitSecurity@0            00408eef f   dmsecure.obj
 0001:00008bb3       _PusrLookupUser@4          00408f13 f   dmsecure.obj
 0001:00008c1c       _DmplAuthenticateUser@16   00408f7c f   dmsecure.obj
 0001:00008cf7       _DmIsSecurityEnabled@4     00409057 f   dmsecure.obj
 0001:00008d1b       _HrDoAddUser@8             0040907b f   dmsecure.obj
 0001:00008def       _DmAddUser@8               0040914f f   dmsecure.obj
 0001:00008e16       _DmRemoveUser@4            00409176 f   dmsecure.obj
 0001:00008e64       _FillAccessPrivSz@8        004091c4 f   dmsecure.obj
 0001:00008edf       _DmplFromSz@4              0040923f f   dmsecure.obj
 0001:00008f4f       _FillUserInfoSz@16         004092af f   dmsecure.obj
 0001:00008faf       _WriteIniSecurity@4        0040930f f   dmsecure.obj
 0001:00009101       _RemoveAllUsers@0          00409461 f   dmsecure.obj
 0001:000091a5       _DmSetUserAccess@8         00409505 f   dmsecure.obj
 0001:000091d0       _DmGetUserAccess@8         00409530 f   dmsecure.obj
 0001:000091fd       _DmWalkUserList@8          0040955d f   dmsecure.obj
 0001:000092a7       _DmCloseCounters@4         00409607 f   dmcount.obj
 0001:000092a7       _DmCloseUserList@4         00409607 f   dmsecure.obj
 0001:000092af       _DmEnableSecurity@4        0040960f f   dmsecure.obj
 0001:000092ca       _HrAddUserCommand@16       0040962a f   dmsecure.obj
 0001:00009358       _FPrintNotifySock@8        004096b8 f   dmnotify.obj
 0001:0000938d       _WriteIniNotifiers@4       004096ed f   dmnotify.obj
 0001:000093f8       _UnNotifyAt@8              00409758 f   dmnotify.obj
 0001:00009420       _FEnsureIPReady@4          00409780 f   dmnotify.obj
 0001:00009451       _SendDebugStrs@8           004097b1 f   dmnotify.obj
 0001:00009688       _GetModLoadSz@8            004099e8 f   dmnotify.obj
 0001:000096de       _GetSectLoadSz@8           00409a3e f   dmnotify.obj
 0001:00009713       _FGetNotifySz@12           00409a73 f   dmnotify.obj
 0001:0000996a       _EnterSessionList@4        00409cca f   dmnotify.obj
 0001:000099ce       _LeaveSessionList@0        00409d2e f   dmnotify.obj
 0001:00009ab4       _NotifyLocalComponents@8   00409e14 f   dmnotify.obj
 0001:00009b20       _NotifyComponents@8        00409e80 f   dmnotify.obj
 0001:00009d04       _FStartThread@12           0040a064 f   dmnotify.obj
 0001:00009d88       _EnterDebuggerDpc@16       0040a0e8 f   dmnotify.obj
 0001:00009d9a       _EnterDebugger@0           0040a0fa f   dmnotify.obj
 0001:00009de1       _TrapHandler@4             0040a141 f   dmnotify.obj
 0001:0000a47f       _DmTrapHandler@20          0040a7df f   dmnotify.obj
 0001:0000a4b1       _DmOpenNotificationSession@8 0040a811 f   dmnotify.obj
 0001:0000a536       _DmCloseNotificationSession@4 0040a896 f   dmnotify.obj
 0001:0000a576       _DmRegisterNotificationProcessor@12 0040a8d6 f   dmnotify.obj
 0001:0000a6be       _DmSendNotificationString@4 0040aa1e f   dmnotify.obj
 0001:0000a7b7       _ClockInt@4                0040ab17 f   dmnotify.obj
 0001:0000a7c3       @CtxSwap@8                 0040ab23 f   dmnotify.obj
 0001:0000a7db       _PrepareToReboot@0         0040ab3b f   dmnotify.obj
 0001:0000a839       _ReportDoubleFault@0       0040ab99 f   dmnotify.obj
 0001:0000a8ba       _CanDebugDF@4              0040ac1a f   dmnotify.obj
 0001:0000a989       _TellDebugger@8            0040ace9 f   dmnotify.obj
 0001:0000aa3d       _InitNotifications@0       0040ad9d f   dmnotify.obj
 0001:0000aaeb       _FAddNotifySock@4          0040ae4b f   dmnotify.obj
 0001:0000ab3e       _FConvertToNotifySock@4    0040ae9e f   dmnotify.obj
 0001:0000ab87       _SockCreateNotify@12       0040aee7 f   dmnotify.obj
 0001:0000aca1       _FNotifyAt@16              0040b001 f   dmnotify.obj
 0001:0000ad73       _FNotifyAtCmd@12           0040b0d3 f   dmnotify.obj
 0001:0000ae2d       _EnsurePersistentSockets@0 0040b18d f   dmnotify.obj
 0001:0000b00e       _ProcessDeferredNotifications@4 0040b36e f   dmnotify.obj
 0001:0000b036       _SetupKernelNotifier@8     0040b396 f   dmnotify.obj
 0001:0000b091       _DmNotify@12               0040b3f1 f   dmnotify.obj
 0001:0000b1fc       _InitBreakpoints@0         0040b55c f   dmbreak.obj
 0001:0000b219       _DoEnableBreak@8           0040b579 f   dmbreak.obj
 0001:0000b281       _DoDisableBreak@8          0040b5e1 f   dmbreak.obj
 0001:0000b2e4       _FFindBreak@16             0040b644 f   dmbreak.obj
 0001:0000b47d       _FIsBreakpoint@4           0040b7dd f   dmbreak.obj
 0001:0000b497       _EnableBreakpointsInRange@12 0040b7f7 f   dmbreak.obj
 0001:0000b521       _DisableBreakpointsInRange@8 0040b881 f   dmbreak.obj
 0001:0000b59a       _FGetMemory@8              0040b8fa f   dmbreak.obj
 0001:0000b609       _FSetMemory@8              0040b969 f   dmbreak.obj
 0001:0000b685       _FAddBreakpoint@4          0040b9e5 f   dmbreak.obj
 0001:0000b74f       _DmSetBreakpoint@4         0040baaf f   dmbreak.obj
 0001:0000b769       _FRemoveBreakpoint@4       0040bac9 f   dmbreak.obj
 0001:0000b7e4       _DmRemoveBreakpoint@4      0040bb44 f   dmbreak.obj
 0001:0000b7fe       _RemoveAllBreakpoints@0    0040bb5e f   dmbreak.obj
 0001:0000b855       _DisableBreakpoint@4       0040bbb5 f   dmbreak.obj
 0001:0000b87e       _SetHwbp@4                 0040bbde f   dmbreak.obj
 0001:0000b8e7       _SyncHwbps@0               0040bc47 f   dmbreak.obj
 0001:0000b918       _DmSetDataBreakpoint@12    0040bc78 f   dmbreak.obj
 0001:0000b9db       _DmIsBreakpoint@8          0040bd3b f   dmbreak.obj
 0001:0000ba39       _FMatchDataBreak@8         0040bd99 f   dmbreak.obj
 0001:0000ba7d       _DoStopGo@4                0040bddd f   dmbreak.obj
 0001:0000bb35       _DoContinue@8              0040be95 f   dmbreak.obj
 0001:0000bb97       _DmGo@0                    0040bef7 f   dmbreak.obj
 0001:0000bbad       _DmStop@0                  0040bf0d f   dmbreak.obj
 0001:0000bbc3       _DoHalt@0                  0040bf23 f   dmbreak.obj
 0001:0000bc90       _SetupHalt@4               0040bff0 f   dmbreak.obj
 0001:0000bcb0       _DmContinueThread@8        0040c010 f   dmbreak.obj
 0001:0000bd0f       _PrepareToStop@0           0040c06f f   dmbreak.obj
 0001:0000bd3a       _FStopAtException@0        0040c09a f   dmbreak.obj
 0001:0000bdab       _DmSetupFunctionCall@4     0040c10b f   dmbreak.obj
 0001:0000be4b       _DwPreFuncCall@4           0040c1ab f   dmbreak.obj
 0001:0000be70       _PostFuncCall@4            0040c1d0 f   dmbreak.obj
 0001:0000be75       _ExceptionsToKd@0          0040c1d5 f   dmbreak.obj
 0001:0000bf06       _ResumeAfterBreakpoint@4   0040c266 f   dmbreak.obj
 0001:0000bf94       _FBreakTrace@4             0040c2f4 f   dmbreak.obj
 0001:0000bfca       _DmGetThreadList@8         0040c32a f   dmbreak.obj
 0001:0000c075       _DmIsThreadStopped@8       0040c3d5 f   dmbreak.obj
 0001:0000c1bd       _DmGetThreadContext@8      0040c51d f   dmbreak.obj
 0001:0000c37d       _DmSetThreadContext@8      0040c6dd f   dmbreak.obj
 0001:0000c4d7       _DmGetThreadInfo@8         0040c837 f   dmbreak.obj
 0001:0000c54f       _DmSetInitialBreakpoint@0  0040c8af f   dmbreak.obj
 0001:0000c56b       _DmStopOn@8                0040c8cb f   dmbreak.obj
 0001:0000c590       _DmReboot@4                0040c8f0 f   dmbreak.obj
 0001:0000c5e6       _DmSuspendThread@4         0040c946 f   dmbreak.obj
 0001:0000c621       _DmResumeThread@4          0040c981 f   dmbreak.obj
 0001:0000c65c       _DmGetXtlData@4            0040c9bc f   dmbreak.obj
 0001:0000c686       _DmHaltThread@4            0040c9e6 f   dmbreak.obj
 0001:0000c714       _InitLoader@0              0040ca74 f   dmmodule.obj
 0001:0000c720       _DmExFreePool@4            0040ca80 f   dmmodule.obj
 0001:0000c726       _PldteGetModule@8          0040ca86 f   dmmodule.obj
 0001:0000c7bf       _DmGetMemory@16            0040cb1f f   dmmodule.obj
 0001:0000c851       _DmSetMemory@16            0040cbb1 f   dmmodule.obj
 0001:0000c8e7       _FixupBistroImage@0        0040cc47 f   dmmodule.obj
 0001:0000c93b       _DwXmhFlags@4              0040cc9b f   dmmodule.obj
 0001:0000c978       _DmWalkLoadedModules@8     0040ccd8 f   dmmodule.obj
 0001:0000ca78       _DmCloseLoadedModules@4    0040cdd8 f   dmmodule.obj
 0001:0000ca8e       _RewindDmws@4              0040cdee f   dmmodule.obj
 0001:0000cada       _DmslFromXsh@8             0040ce3a f   dmmodule.obj
 0001:0000cb37       _DmWalkModuleSections@12   0040ce97 f   dmmodule.obj
 0001:0000cc3b       _DmCloseModuleSections@4   0040cf9b f   dmmodule.obj
 0001:0000cc53       _DmGetModuleLongName@12    0040cfb3 f   dmmodule.obj
 0001:0000ccc6       _DmGetXbeInfo@8            0040d026 f   dmmodule.obj
 0001:0000cdd5       _FResolveImport@20         0040d135 f   dmmodule.obj
 0001:0000cf21       _FFinishImageLoad@12       0040d281 f   dmmodule.obj
 0001:0000d086       _UnloadReferencedModules@4 0040d3e6 f   dmmodule.obj
 0001:0000d0ba       _DmUnloadExtension@4       0040d41a f   dmmodule.obj
 0001:0000d152       _DmGetProcAddress@12       0040d4b2 f   dmmodule.obj
 0001:0000d1ab       _FResolveImageImports@12   0040d50b f   dmmodule.obj
 0001:0000d368       _FFixupXbdm@8              0040d6c8 f   dmmodule.obj
 0001:0000d3f4       _StLoadImage@12            0040d754 f   dmmodule.obj
 0001:0000d63a       _DmLoadExtension@12        0040d99a f   dmmodule.obj
 0001:0000d7bd       _FGetCounterValue@12       0040db1d f   dmcount.obj
 0001:0000d83f       _RefreshCounter@4          0040db9f f   dmcount.obj
 0001:0000d914       _CounterDpc@16             0040dc74 f   dmcount.obj
 0001:0000da3b       _DmRegisterPerformanceCounter@12 0040dd9b f   dmcount.obj
 0001:0000db4d       _DmOpenPerformanceCounter@8 0040dead f   dmcount.obj
 0001:0000dbb9       _DmQueryPerformanceCounterHandle@12 0040df19 f   dmcount.obj
 0001:0000de5b       _DmClosePerformanceCounter@4 0040e1bb f   dmcount.obj
 0001:0000de7e       _DmWalkPerformanceCounters@8 0040e1de f   dmcount.obj
 0001:0000df7a       _GPUPerf@4                 0040e2da f   dmcount.obj
 0001:0000dffd       _DmEnableGPUCounter@4      0040e35d f   dmcount.obj
 0001:0000e062       _InitCounters@0            0040e3c2 f   dmcount.obj
 0001:0000e191       _DmUnregisterPerformanceCounter@4 0040e4f1 f   dmcount.obj
 0001:0000e218       _QueuePob@4                0040e578 f   dmprofil.obj
 0001:0000e2a6       _DeletePob@4               0040e606 f   dmprofil.obj
 0001:0000e327       _DmStartProfile@12         0040e687 f   dmprofil.obj
 0001:0000e3f4       _DmStopProfile@4           0040e754 f   dmprofil.obj
 0001:0000e42a       _ProfInt@4                 0040e78a f   dmprofil.obj
 0001:0000e4c2       _MapDebugDrive@8           0040e822 f   dmfile.obj
 0001:0000e530       _FObNameToFileName@12      0040e890 f   dmfile.obj
 0001:0000e5d9       _FFileNameToObName@12      0040e939 f   dmfile.obj
 0001:0000e6a5       _FCreateFile@32            0040ea05 f   dmfile.obj
 0001:0000e716       _QueueDmpp@4               0040ea76 f   dmpool.obj
 0001:0000e7b4       _DmpFreePoolMemory@8       0040eb14 f   dmpool.obj
 0001:0000e850       _DmpAllocatePoolMemory@4   0040ebb0 f   dmpool.obj
 0001:0000e957       _DmpAllocatePoolPages@4    0040ecb7 f   dmpool.obj
 0001:0000e99a       _ExpRemovePoolTracker@8    0040ecfa f   dmpool.obj
 0001:0000ea33       _ExpFindAndRemoveTagBigPages@4 0040ed93 f   dmpool.obj
 0001:0000eab2       _DmFreePool@4              0040ee12 f   dmpool.obj
 0001:0000ec7a       _ExpInsertPoolTracker@8    0040efda f   dmpool.obj
 0001:0000ee83       _ExpAddTagForBigPages@12   0040f1e3 f   dmpool.obj
 0001:0000efcd       _InitPool@0                0040f32d f   dmpool.obj
 0001:0000f103       _DmAllocatePoolWithTag@8   0040f463 f   dmpool.obj
 0001:0000f332       _DmAllocatePool@4          0040f692 f   dmpool.obj
 0001:0000f343       __CAP_Start_Profiling@8    0040f6a3 f   dmcap.obj
 0001:0000f37c       __CAP_End_Profiling@4      0040f6dc f   dmcap.obj
 0001:0000f3b2       __CAP_Enter_Function@4     0040f712 f   dmcap.obj
 0001:0000f3e8       __CAP_Exit_Function@4      0040f748 f   dmcap.obj
 0001:0000f420       __penter                   0040f780 f   dmcap.obj
 0001:0000f457       __pexit                    0040f7b7 f   dmcap.obj
 0001:0000f490       _DmProfileEmitControlRecord@8 0040f7f0 f   dmcap.obj
 0001:0000f4cb       @DmProfileThreadSwitchNotifyCallback@8 0040f82b f   dmcap.obj
 0001:0000f4ed       @DmProfileDpcDispatchNotifyCallback@8 0040f84d f   dmcap.obj
 0001:0000f4f8       _DmCapControl@8            0040f858 f   dmcap.obj
 0001:0000f72b       _DmProfileControl@8        0040fa8b f   dmcap.obj
 0001:0000f742       _SetLastError@4            0040faa2 f   api32.obj
 0001:0000f757       _GetLastError@0            0040fab7 f   api32.obj
 0001:0000f766       _LocalAlloc@8              0040fac6 f   api32.obj
 0001:0000f7ba       _LocalFree@4               0040fb1a f   api32.obj
 0001:0000f80a       _SleepEx@8                 0040fb6a f   api32.obj
 0001:0000f868       __DmUnhandledException@4   0040fbc8 f   api32.obj
 0001:0000f87f       __DmThreadStartup@8        0040fbdf f   api32.obj
 0001:0000f8bf       _CreateThread@24           0040fc1f f   api32.obj
 0001:0000f915       _CloseHandle@4             0040fc75 f   api32.obj
 0001:0000f944       _Sleep@4                   0040fca4 f   api32.obj
 0001:0000f952       _Crc32@12                  0040fcb2 f   crc.obj
 0001:0000f97f       _FlashGetStatus@12         0040fcdf f   flash.obj
 0001:0000f9f9       _FlashResetDevice@0        0040fd59 f   flash.obj
 0001:0000fa29       _FlashDetectDevice@0       0040fd89 f   flash.obj
 0001:0000fb35       _FlashEraseChip@4          0040fe95 f   flash.obj
 0001:0000fc49       _FlashProgramImage@8       0040ffa9 f   flash.obj
 0001:0000fd69       @FlashReadMSR@4            004100c9 f   flash.obj
 0001:0000fd6c       @FlashWriteMSR@12          004100cc f   flash.obj
 0001:0000fd79       _FlashChangeRomCaching@4   004100d9 f   flash.obj
 0001:0000fe2c       _FlashKernelImage@20       0041018c f   flash.obj
 0001:0000ffa8       _ReplaceFile@8             00410308 f   sysfileupd.obj
 0001:0001004a       _HrReceiveSystemFile@12    004103aa f   sysfileupd.obj
 0001:000101da       _CreateDirectoryFromPath@4 0041053a f   sysfileupd.obj
 0001:00010262       _HrUpdateSystemFile@16     004105c2 f   sysfileupd.obj
 0001:000104e7       _RtlImageNtHeader@4        00410847 f   xbdmrtl:imagedir.obj
 0001:00010526       _RtlSectionTableFromVirtualAddress@12 00410886 f   xbdmrtl:imagedir.obj
 0001:00010561       _RtlAddressInSectionTable@12 004108c1 f   xbdmrtl:imagedir.obj
 0001:0001058c       _RtlpImageDirectoryEntryToData32@20 004108ec f   xbdmrtl:imagedir.obj
 0001:000105e8       _RtlImageDirectoryEntryToData@16 00410948 f   xbdmrtl:imagedir.obj
 0001:00010626       _LdrProcessRelocationBlock@16 00410986 f   xbdmrtl:ldrreloc.obj
 0001:000106a2       _LdrRelocateImage@20       00410a02 f   xbdmrtl:ldrreloc.obj
 0001:00010710       _XWriteTitleInfoNoReboot@20 00410a70 f   dmxapi:launch.obj
 0001:000107e3       _XapiFormatFATVolumeEx@8   00410b43 f   dmxapi:format.obj
 0001:00010af9       _XapiFormatFATVolume@4     00410e59 f   dmxapi:format.obj
 0001:00010b0a       _IsBadReadPtr@8            00410e6a f   dmxapi:process.obj
 0001:00010b6f       _IsBadWritePtr@8           00410ecf f   dmxapi:process.obj
 0001:00010bd8       _lstrcpynA@12              00410f38 f   dmxapi:lcompata.obj
 0001:00010c3d       _XapiSetLastNTError@4      00410f9d f   dmxapi:error.obj
 0001:00010c60       @RtlFindFirstSetRightMember@4 00410fc0 f   xapirtl:bitmapa.obj
 0001:00010c70       _memmove                   00410fd0 f   libcntpr:memmove.obj
 0001:00010fa5       _sprintf                   00411305 f   libcntpr:sprintf.obj
 0001:00011000       _strncpy                   00411360 f   libcntpr:strncpy.obj
 0001:00011100       _strrchr                   00411460 f   libcntpr:strrchr.obj
 0001:00011127       __snprintf                 00411487 f   libcntpr:snprintf.obj
 0001:00011180       __allmul                   004114e0 f   libcntpr:llmul.obj
 0001:000111d0       _strchr                    00411530 f   libcntpr:strchr.obj
 0001:000111d6       ___from_strstr_to_strchr   00411536     libcntpr:strchr.obj
 0001:0001128c       __SEH_prolog               004115ec f   libcntpr:sehprolg.obj
 0001:000112c5       __SEH_epilog               00411625 f   libcntpr:sehprolg.obj
 0001:000112e0       __except_handler3          00411640 f   libcntpr:exsup3.obj
 0001:0001139d       __seh_longjmp_unwind@4     004116fd f   libcntpr:exsup3.obj
 0001:000113b8       __strnicmp                 00411718 f   libcntpr:strnicmp.obj
 0001:000113cb       _wcschr                    0041172b f   libcntpr:wcschr.obj
 0001:000113f0       __alldiv                   00411750 f   libcntpr:lldiv.obj
 0001:0001149a       __flsbuf                   004117fa f   libcntpr:_flsbuf.obj
 0001:00011538       __output                   00411898 f   libcntpr:output.obj
 0001:00011ba0       __global_unwind2           00411f00 f   libcntpr:exsup.obj
 0001:00011be2       __local_unwind2            00411f42 f   libcntpr:exsup.obj
 0001:00011c3a       __NLG_Return2              00411f9a     libcntpr:exsup.obj
 0001:00011c4a       __abnormal_termination     00411faa f   libcntpr:exsup.obj
 0001:00011c6d       __NLG_Notify1              00411fcd f   libcntpr:exsup.obj
 0001:00011c76       __NLG_Notify               00411fd6 f   libcntpr:exsup.obj
 0001:00011c89       __NLG_Dispatch             00411fe9     libcntpr:exsup.obj
 0001:00011c90       ___ascii_strnicmp          00411ff0 f   libcntpr:_strnicm.obj
 0001:00011cf0       ___ascii_stricmp           00412050 f   libcntpr:_stricmp.obj
 0001:00011d3a       _wctomb                    0041209a f   libcntpr:wctomb.obj
 0001:00011d70       __aulldvrm                 004120d0 f   libcntpr:ulldvrm.obj
 0001:00011e06       _ExSaveNonVolatileSetting@16 00412166 f   xboxkrnl:xboxkrnl.exe
 0001:00011e0c       _DbgPrint                  0041216c f   xboxkrnl:xboxkrnl.exe
 0001:00011e12       _PsSetCreateThreadNotifyRoutine@4 00412172 f   xboxkrnl:xboxkrnl.exe
 0001:00011e18       _ExQueryNonVolatileSetting@20 00412178 f   xboxkrnl:xboxkrnl.exe
 0001:00011e1e       _XcModExp@20               0041217e f   xboxkrnl:xboxkrnl.exe
 0001:00011e24       _KeSuspendThread@4         00412184 f   xboxkrnl:xboxkrnl.exe
 0001:00011e2a       _KeResumeThread@4          0041218a f   xboxkrnl:xboxkrnl.exe
 0001:00011e30       _XcRC4Crypt@12             00412190 f   xboxkrnl:xboxkrnl.exe
 0001:00011e36       _XcRC4Key@12               00412196 f   xboxkrnl:xboxkrnl.exe
 0001:00011e3c       _XcSHAFinal@8              0041219c f   xboxkrnl:xboxkrnl.exe
 0001:00011e42       _XcSHAUpdate@12            004121a2 f   xboxkrnl:xboxkrnl.exe
 0001:00011e48       _XcSHAInit@4               004121a8 f   xboxkrnl:xboxkrnl.exe
 0001:00011e4e       _XcBlockCryptCBC@28        004121ae f   xboxkrnl:xboxkrnl.exe
 0001:00011e54       _XcKeyTable@12             004121b4 f   xboxkrnl:xboxkrnl.exe
 0001:00011e5a       _XcDESKeyParity@8          004121ba f   xboxkrnl:xboxkrnl.exe
 0001:00011e60       _XcHMAC@28                 004121c0 f   xboxkrnl:xboxkrnl.exe
 0001:00011e66       _RtlUnwind@16              004121c6 f   xboxkrnl:xboxkrnl.exe
 0002:00000000       ?SockCountSendTotal@@YGIPAU_WSABUF@@I@Z 004121e0 f   xnetm:sock.obj
 0002:00000019       _WSAGetLastError@0         004121f9 f   xnetm:sock.obj
 0002:0000001e       ___WSAFDIsSet@8            004121fe f   xnetm:sock.obj
 0002:00000049       ?Lock@CSocket@@SGPAV1@I@Z  00412229 f   xnetm:sock.obj
 0002:000000a1       ?SockInit@CXnSock@@QAEJPAUXNetInitParams@@@Z 00412281 f   xnetm:sock.obj
 0002:000000e9       ?SetFlagsAndOr@CSocket@@QAEXKK@Z 004122c9 f   xnetm:sock.obj
 0002:00000121       ?SockAlloc@CXnSock@@AAEPAVCSocket@@HH@Z 00412301 f   xnetm:sock.obj
 0002:0000028f       ?SockFree@CXnSock@@AAEXPAVCSocket@@@Z 0041246f f   xnetm:sock.obj
 0002:000002b1       ?SockReleaseSendBuf@CXnSock@@AAEXPAVCSendBuf@@@Z 00412491 f   xnetm:sock.obj
 0002:000002cc       ?SockFlushRecvBuffers@CXnSock@@AAEXPAVCSocket@@@Z 004124ac f   xnetm:sock.obj
 0002:000002fc       ?shutdown@CXnSock@@QAEHIH@Z 004124dc f   xnetm:sock.obj
 0002:00000398       ?ioctlsocket@CXnSock@@QAEHIJPAK@Z 00412578 f   xnetm:sock.obj
 0002:00000460       ?SockUpdateBufferSize@CXnSock@@AAEJPAVCSocket@@HH@Z 00412640 f   xnetm:sock.obj
 0002:000004bc       ?getpeername@CXnSock@@QAEHIPAUsockaddr@@PAH@Z 0041269c f   xnetm:sock.obj
 0002:00000548       ?SockBind@CXnSock@@AAEJPAVCSocket@@UCIpPort@@@Z 00412728 f   xnetm:sock.obj
 0002:0000066d       ?listen@CXnSock@@QAEHIH@Z  0041284d f   xnetm:sock.obj
 0002:000006ef       ?SockLockSelectSockets@CXnSock@@AAEHPAUfd_set@@PAU_SELECTINFO@1@HH@Z 004128cf f   xnetm:sock.obj
 0002:000007cd       ?SockCheckSelectEvents@CXnSock@@AAEHPAVCSocket@@HH@Z 004129ad f   xnetm:sock.obj
 0002:000008d0       ?RecvReqEnqueue@CXnSock@@AAEJPAVCSocket@@PAVCRecvReq@@@Z 00412ab0 f   xnetm:sock.obj
 0002:00000945       ?SockQueueOverlappedSend@CXnSock@@AAEJPAVCSocket@@PAVCSendReq@@@Z 00412b25 f   xnetm:sock.obj
 0002:00000a11       _htonl@4                   00412bf1 f   xnetm:sock.obj
 0002:00000a11       _ntohl@4                   00412bf1 f   xnetm:sock.obj
 0002:00000a3b       _htons@4                   00412c1b f   xnetm:sock.obj
 0002:00000a4f       ?SockWaitForEvent@CXnSock@@AAEJPAVCSocket@@HI@Z 00412c2f f   xnetm:sock.obj
 0002:00000acf       ?SockReqComplete@CXnSock@@AAEXPAVCSocket@@PAVCSockReq@@J@Z 00412caf f   xnetm:sock.obj
 0002:00000b21       ?SockFindMatch@CXnSock@@AAEPAVCSocket@@UCIpPort@@UCIpAddr@@0E@Z 00412d01 f   xnetm:sock.obj
 0002:00000bab       ?SockReset@CXnSock@@AAEXUCIpAddr@@@Z 00412d8b f   xnetm:sock.obj
 0002:00000c1d       ?socket@CXnSock@@QAEIHHH@Z 00412dfd f   xnetm:sock.obj
 0002:00000d10       ?SockCleanup@CXnSock@@AAEXPAVCSocket@@@Z 00412ef0 f   xnetm:sock.obj
 0002:00000d84       ?setsockopt@CXnSock@@QAEHIHHPBDH@Z 00412f64 f   xnetm:sock.obj
 0002:00000f79       ?bind@CXnSock@@QAEHIPBUsockaddr@@H@Z 00413159 f   xnetm:sock.obj
 0002:00000ffc       ?connect@CXnSock@@QAEHIPBUsockaddr@@H@Z 004131dc f   xnetm:sock.obj
 0002:000010e4       ?accept@CXnSock@@QAEIIPAUsockaddr@@PAH@Z 004132c4 f   xnetm:sock.obj
 0002:00001205       ?select@CXnSock@@QAEHHPAUfd_set@@00PBUtimeval@@@Z 004133e5 f   xnetm:sock.obj
 0002:000015a8       ?SockRead@CXnSock@@AAEJPAVCSocket@@PAVCRecvReq@@@Z 00413788 f   xnetm:sock.obj
 0002:00001764       ?SockSend@CXnSock@@AAEJPAVCSocket@@PAVCSendReq@@@Z 00413944 f   xnetm:sock.obj
 0002:0000187d       ?SockClose@CXnSock@@AAEJPAVCSocket@@H@Z 00413a5d f   xnetm:sock.obj
 0002:0000191d       ?recv@CXnSock@@QAEHIPADHH@Z 00413afd f   xnetm:sock.obj
 0002:000019ad       ?WSARecvFrom@CXnSock@@QAEHIPAU_WSABUF@@KPAK1PAUsockaddr@@PAHPAU_OVERLAPPED@@P6GXKK4K@Z@Z 00413b8d f   xnetm:sock.obj
 0002:00001a6a       ?send@CXnSock@@QAEHIPBDHH@Z 00413c4a f   xnetm:sock.obj
 0002:00001afe       ?WSASend@CXnSock@@QAEHIPAU_WSABUF@@KPAKKPAU_OVERLAPPED@@P6GXKK2K@Z@Z 00413cde f   xnetm:sock.obj
 0002:00001b98       ?WSASendTo@CXnSock@@QAEHIPAU_WSABUF@@KPAKKPBUsockaddr@@HPAU_OVERLAPPED@@P6GXKK3K@Z@Z 00413d78 f   xnetm:sock.obj
 0002:00001ca2       ?SockShutdown@CXnSock@@QAEXXZ 00413e82 f   xnetm:sock.obj
 0002:00001cf2       ?closesocket@CXnSock@@QAEHI@Z 00413ed2 f   xnetm:sock.obj
 0002:00001d81       ?recvfrom@CXnSock@@QAEHIPADHHPAUsockaddr@@PAH@Z 00413f61 f   xnetm:sock.obj
 0002:00001dc2       ?sendto@CXnSock@@QAEHIPBDHHPBUsockaddr@@H@Z 00413fa2 f   xnetm:sock.obj
 0002:00001e02       ?SockTerm@CXnSock@@QAEXXZ  00413fe2 f   xnetm:sock.obj
 0002:00001e3f       ?XNetRandom@CXn@@QAEHPAEI@Z 0041401f f   xnetm:xnet.obj
 0002:00001e5c       ?XNetInAddrToString@CXn@@QAEHUin_addr@@PADH@Z 0041403c f   xnetm:xnet.obj
 0002:00001e72       ?XNetGetTitleXnAddr@CXn@@QAEKPAUXNADDR@@@Z 00414052 f   xnetm:xnet.obj
 0002:00001e81       ?XNetGetDebugXnAddr@CXn@@QAEKPAUXNADDR@@@Z 00414061 f   xnetm:xnet.obj
 0002:00001e90       _XNetRandom@8              00414070 f   xnetm:xnet.obj
 0002:00001e9b       _XNetInAddrToString@12     0041407b f   xnetm:xnet.obj
 0002:00001ea6       _XNetGetTitleXnAddr@4      00414086 f   xnetm:xnet.obj
 0002:00001eb1       _XNetGetDebugXnAddr@4      00414091 f   xnetm:xnet.obj
 0002:00001ebc       _socket@12                 0041409c f   xnetm:xnet.obj
 0002:00001ec7       _closesocket@4             004140a7 f   xnetm:xnet.obj
 0002:00001ed2       _shutdown@8                004140b2 f   xnetm:xnet.obj
 0002:00001edd       _ioctlsocket@12            004140bd f   xnetm:xnet.obj
 0002:00001ee8       _setsockopt@20             004140c8 f   xnetm:xnet.obj
 0002:00001ef7       _getpeername@12            004140d7 f   xnetm:xnet.obj
 0002:00001f02       _bind@12                   004140e2 f   xnetm:xnet.obj
 0002:00001f0d       _connect@12                004140ed f   xnetm:xnet.obj
 0002:00001f18       _listen@8                  004140f8 f   xnetm:xnet.obj
 0002:00001f23       _accept@12                 00414103 f   xnetm:xnet.obj
 0002:00001f2e       _select@20                 0041410e f   xnetm:xnet.obj
 0002:00001f3d       _recv@16                   0041411d f   xnetm:xnet.obj
 0002:00001f48       _recvfrom@24               00414128 f   xnetm:xnet.obj
 0002:00001f57       _send@16                   00414137 f   xnetm:xnet.obj
 0002:00001f62       _WSASend@28                00414142 f   xnetm:xnet.obj
 0002:00001f71       _sendto@24                 00414151 f   xnetm:xnet.obj
 0002:00001f80       ??0CIpAddr@@QAE@XZ         00414160 f i xnetm:sock.obj
 0002:00001f80       ??0CArpEntry@CXnEnet@@QAE@XZ 00414160 f i xnetm:xnet.obj
 0002:00001f83       ??_H@YGXPAXIHP6EPAX0@Z@Z   00414163 f i xnetm:xnet.obj
 0002:00001fa5       ??0CXn@@QAE@XZ             00414185 f i xnetm:xnet.obj
 0002:00001ffd       _XnInit@24                 004141dd f   xnetm:xnet.obj
 0002:00002214       _XNetStartup@4             004143f4 f   xnetm:xnet.obj
 0002:0000222b       _WSAStartup@8              0041440b f   xnetm:xnet.obj
 0002:00002246       ?RandInit@CXnBase@@AAEXPAUXNetInitParams@@@Z 00414426 f   xnetm:base.obj
 0002:000022e8       ?InsertHead@CPacketQueue@@QAEXPAVCPacket@@@Z 004144c8 f   xnetm:base.obj
 0002:000022fd       ?InsertTail@CPacketQueue@@QAEXPAVCPacket@@@Z 004144dd f   xnetm:base.obj
 0002:00002319       ?RemoveHead@CPacketQueue@@QAEPAVCPacket@@XZ 004144f9 f   xnetm:base.obj
 0002:0000232d       ?Dequeue@CPacketQueue@@QAEXPAVCPacket@@@Z 0041450d f   xnetm:base.obj
 0002:00002367       ?XnInAddrToString@@YGXUin_addr@@PADH@Z 00414547 f   xnetm:base.obj
 0002:000023ec       ?TimerSet@CXnBase@@QAEXPAVCTimer@@K@Z 004145cc f   xnetm:base.obj
 0002:00002451       ?TimerSetRelative@CXnBase@@QAEKPAVCTimer@@K@Z 00414631 f   xnetm:base.obj
 0002:00002472       ?PoolAlloc@CXnBase@@QAEPAXIK@Z 00414652 f   xnetm:base.obj
 0002:00002572       ?PoolAllocZ@CXnBase@@QAEPAXIK@Z 00414752 f   xnetm:base.obj
 0002:000025a4       ?PoolFree@CXnBase@@QAEXPAX@Z 00414784 f   xnetm:base.obj
 0002:0000265a       ?Rand@CXnBase@@QAEXPAEI@Z  0041483a f   xnetm:base.obj
 0002:00002684       ?RandLong@CXnBase@@QAEKXZ  00414864 f   xnetm:base.obj
 0002:00002698       ?PacketFree@CXnBase@@QAEXPAVCPacket@@@Z 00414878 f   xnetm:base.obj
 0002:000026b3       ?GetHdr@CPacket@@QAEPAXH@Z 00414893 f   xnetm:base.obj
 0002:000026e9       ?InsertHead@CPacketQueue@@QAEXPAV1@@Z 004148c9 f   xnetm:base.obj
 0002:00002712       ?Complete@CPacketQueue@@QAEXPAVCXnBase@@@Z 004148f2 f   xnetm:base.obj
 0002:0000272f       ?Discard@CPacketQueue@@QAEXPAVCXnBase@@@Z 0041490f f   xnetm:base.obj
 0002:0000274e       ?DefaultMask@CIpAddr@@QBE?AU1@XZ 0041492e f   xnetm:base.obj
 0002:000027b0       ?TimerPush@CXnBase@@AAEXXZ 00414990 f   xnetm:base.obj
 0002:00002807       ?BaseStart@CXnBase@@QAEXXZ 004149e7 f   xnetm:base.obj
 0002:0000282d       ?BaseStop@CXnBase@@QAEXXZ  00414a0d f   xnetm:base.obj
 0002:00002865       ?BaseTerm@CXnBase@@QAEXXZ  00414a45 f   xnetm:base.obj
 0002:00002896       ?PacketAlloc@CXnBase@@QAEPAVCPacket@@KIIIP8CXnVoid@@AEXPAV2@@Z@Z 00414a76 f   xnetm:base.obj
 0002:0000298a       ?IsValidUnicast@CIpAddr@@QBEHXZ 00414b6a f   xnetm:base.obj
 0002:000029b3       ?TimerDpc@CXnBase@@CGXPAU_KDPC@@PAX11@Z 00414b93 f   xnetm:base.obj
 0002:000029bf       ?BaseInit@CXnBase@@QAEJPAUXNetInitParams@@@Z 00414b9f f   xnetm:base.obj
 0002:00002b6a       ?HalQueryTsc@@YGXPAT_LARGE_INTEGER@@@Z 00414d4a f   xnetm:halx.obj
 0002:00002b6f       ?Add@CRandBytes@@QAEXPAXI@Z 00414d4f f   xnetm:halx.obj
 0002:00002b9e       ?SetInitFlag@CXnHal@@QAEXK@Z 00414d7e f   xnetm:halx.obj
 0002:00002bcd       ?HalRandGather@CXnHal@@QAEIPAEI@Z 00414dad f   xnetm:halx.obj
 0002:00002cda       ?FragFree@CXnIp@@AAEXPAVCPacket@@@Z 00414eba f   xnetm:ip.obj
 0002:00002d0e       ?FragTimer@CXnIp@@AAEXPAVCTimer@@@Z 00414eee f   xnetm:ip.obj
 0002:00002d1e       ?RouteRelease@CXnIp@@QAEXPAVCRouteEntry@@@Z 00414efe f   xnetm:ip.obj
 0002:00002d4e       ?KeyRegLookup@CXnIp@@AAEPAUCKeyReg@1@PBUXNKID@@@Z 00414f2e f   xnetm:ip.obj
 0002:00002d81       ?CryptDes@CXnIp@@AAEXKPAEI00I@Z 00414f61 f   xnetm:ip.obj
 0002:00002dd6       ?SecRegSetKey@CXnIp@@AAEXPAUCSecReg@1@PAEI1I1IH@Z 00414fb6 f   xnetm:ip.obj
 0002:00002e66       ?IpInit@CXnIp@@IAEJPAUXNetInitParams@@@Z 00415046 f   xnetm:ip.obj
 0002:00002f62       ?IpConfig@CXnIp@@IAEHPBUXNetConfigParams@@K@Z 00415142 f   xnetm:ip.obj
 0002:00002f8a       ?IpRecvTcp@CXnIp@@AAEXPAVCPacket@@PAUCIpHdr@@PAUCTcpHdr@@I@Z 0041516a f   xnetm:ip.obj
 0002:00003048       ?IpFillHdr@CXnIp@@QAEXPAVCPacket@@UCIpAddr@@E@Z 00415228 f   xnetm:ip.obj
 0002:000030b5       ?FragTerm@CXnIp@@AAEXXZ    00415295 f   xnetm:ip.obj
 0002:000030d6       ?RouteEntryOrphan@CXnIp@@AAEXPAVCRouteEntry@@@Z 004152b6 f   xnetm:ip.obj
 0002:00003101       ?RouteLookup@CXnIp@@AAEPAVCRouteEntry@@UCIpAddr@@@Z 004152e1 f   xnetm:ip.obj
 0002:00003198       ?RouteAdd@CXnIp@@AAEXUCIpAddr@@00GG@Z 00415378 f   xnetm:ip.obj
 0002:000032b3       ?RouteDelete@CXnIp@@AAEXUCIpAddr@@00@Z 00415493 f   xnetm:ip.obj
 0002:00003307       ?RouteRedirect@CXnIp@@AAEXUCIpAddr@@00@Z 004154e7 f   xnetm:ip.obj
 0002:00003374       ?SecRegLookup@CXnIp@@AAEPAUCSecReg@1@PBUXNADDR@@PBUXNKID@@@Z 00415554 f   xnetm:ip.obj
 0002:000033ca       ?SecRegLookup@CXnIp@@AAEPAUCSecReg@1@K@Z 004155aa f   xnetm:ip.obj
 0002:00003407       ?SecRegSetTicks@CXnIp@@AAEXPAUCSecReg@1@@Z 004155e7 f   xnetm:ip.obj
 0002:00003439       ?SecRegSetOwned@CXnIp@@QAEXUCIpAddr@@@Z 00415619 f   xnetm:ip.obj
 0002:00003472       ?IpDecrypt@CXnIp@@QAEHPAVCPacket@@UCIpAddr@@@Z 00415652 f   xnetm:ip.obj
 0002:00003518       ?IpGetXnAddr@CXnIp@@QAEKPAUXNADDR@@@Z 004156f8 f   xnetm:ip.obj
 0002:000035af       ?IpFillKeyExXbToXb@CXnIp@@AAEXPAUCSecReg@1@PAUCKeyExXbToXb@1@@Z 0041578f f   xnetm:ip.obj
 0002:000036ec       ?IpXmitIp@CXnIp@@AAEXPAVCPacket@@PAPAVCRouteEntry@@@Z 004158cc f   xnetm:ip.obj
 0002:00003865       ?RouteListOrphan@CXnIp@@AAEXXZ 00415a45 f   xnetm:ip.obj
 0002:0000388e       ?SecRegSetIdle@CXnIp@@AAEXPAUCSecReg@1@@Z 00415a6e f   xnetm:ip.obj
 0002:000038f0       ?IpSetAddress@CXnIp@@QAEXUCIpAddr@@0@Z 00415ad0 f   xnetm:ip.obj
 0002:000039a2       ?IpXmitEsp@CXnIp@@AAEXPAVCPacket@@PAUCSecReg@1@PAPAVCRouteEntry@@@Z 00415b82 f   xnetm:ip.obj
 0002:00003ba2       ?IpXmitKeyExXbToXb@CXnIp@@AAEXPAUCSecReg@1@H@Z 00415d82 f   xnetm:ip.obj
 0002:00003c4c       ?IpXmitSecMsg@CXnIp@@AAEXPAUCSecReg@1@GPAXI1I@Z 00415e2c f   xnetm:ip.obj
 0002:00003cfd       ?IpXmitSecMsgDelete@CXnIp@@AAEXPAUCSecReg@1@K@Z 00415edd f   xnetm:ip.obj
 0002:00003d19       ?SecRegFree@CXnIp@@AAEXPAUCSecReg@1@@Z 00415ef9 f   xnetm:ip.obj
 0002:00003d35       ?SecRegShutdown@CXnIp@@QAEXH@Z 00415f15 f   xnetm:ip.obj
 0002:00003d93       ?SecRegProbe@CXnIp@@AAEXXZ 00415f73 f   xnetm:ip.obj
 0002:00003e74       ?IpStop@CXnIp@@IAEXXZ      00416054 f   xnetm:ip.obj
 0002:00003ea9       ?IpRecvSecMsg@CXnIp@@AAEXPAVCPacket@@PAUCSecReg@1@KPAUCSecMsgHdr@@I@Z 00416089 f   xnetm:ip.obj
 0002:00003ee4       ?IpXmitKeyEx@CXnIp@@AAEXPAUCSecReg@1@@Z 004160c4 f   xnetm:ip.obj
 0002:00003f37       ?IpUnregisterKey@CXnIp@@QAEHPBUXNKID@@@Z 00416117 f   xnetm:ip.obj
 0002:00004006       ?SecRegEnqueue@CXnIp@@AAEXPAUCSecReg@1@PAVCPacket@@@Z 004161e6 f   xnetm:ip.obj
 0002:00004027       ?SecRegTimer@CXnIp@@AAEXPAVCTimer@@@Z 00416207 f   xnetm:ip.obj
 0002:00004076       ?IpTerm@CXnIp@@IAEXXZ      00416256 f   xnetm:ip.obj
 0002:0000413b       ?IpXmit@CXnIp@@QAEXPAVCPacket@@PAPAVCRouteEntry@@@Z 0041631b f   xnetm:ip.obj
 0002:000041d3       ?IpFillAndXmit@CXnIp@@QAEXPAVCPacket@@UCIpAddr@@EPAPAVCRouteEntry@@@Z 004163b3 f   xnetm:ip.obj
 0002:0000420b       ?SecRegAlloc@CXnIp@@AAEPAUCSecReg@1@XZ 004163eb f   xnetm:ip.obj
 0002:000042a2       ?SecRegAlloc@CXnIp@@AAEPAUCSecReg@1@PBUXNADDR@@PAUCKeyReg@1@@Z 00416482 f   xnetm:ip.obj
 0002:000042f3       ?SecRegXmitQueue@CXnIp@@AAEXPAUCSecReg@1@@Z 004164d3 f   xnetm:ip.obj
 0002:0000431b       ?IpRecvKeyExXbToXb@CXnIp@@AAEXPAVCPacket@@UCIpAddr@@UCIpPort@@PAUCKeyExXbToXb@1@I@Z 004164fb f   xnetm:ip.obj
 0002:000046a9       ?IpRecvKeyEx@CXnIp@@AAEXPAVCPacket@@UCIpAddr@@UCIpPort@@PAUCKeyExHdr@@I@Z 00416889 f   xnetm:ip.obj
 0002:000046ee       ?IpRecvEsp@CXnIp@@AAEXPAVCPacket@@PAUCIpHdr@@PAUCEspHdr@@I@Z 004168ce f   xnetm:ip.obj
 0002:00004a2d       ?IpRecvUdp@CXnIp@@AAEXPAVCPacket@@PAUCIpHdr@@PAUCUdpHdr@@I@Z 00416c0d f   xnetm:ip.obj
 0002:00004b25       ?IpRecv@CXnIp@@IAEXPAVCPacket@@@Z 00416d05 f   xnetm:ip.obj
 0002:00004cc8       ?FragRecv@CXnIp@@AAEXPAVCPacket@@PAUCIpHdr@@II@Z 00416ea8 f   xnetm:ip.obj
 0002:00004f9b       ?TcpValidateSeqs@CXnSock@@AAEHPAVCTcpSocket@@KKPAK1@Z 0041717b f   xnetm:socktcp.obj
 0002:00004fee       ?DequeueChild@CTcpSocket@@QAEXPAV1@@Z 004171ce f   xnetm:socktcp.obj
 0002:00005012       ?InsertRecvBuf@CSocket@@QAEXPAVCRecvBuf@@0@Z 004171f2 f   xnetm:socktcp.obj
 0002:0000503f       ?TcpSndNxt@CXnSock@@AAEKPAVCTcpSocket@@@Z 0041721f f   xnetm:socktcp.obj
 0002:0000506e       ?TcpSlideRecvWindow@CXnSock@@AAEXPAVCTcpSocket@@I@Z 0041724e f   xnetm:socktcp.obj
 0002:000050ad       ?TcpUpdateRTO@CXnSock@@AAEXPAVCTcpSocket@@@Z 0041728d f   xnetm:socktcp.obj
 0002:00005168       ?TcpCorrectMisorderedSegments@CXnSock@@AAEIPAVCTcpSocket@@KPAVCTcpRecvBuf@@@Z 00417348 f   xnetm:socktcp.obj
 0002:0000521a       ?TcpBufferMisorderedSegment@CXnSock@@AAEXPAVCTcpSocket@@IPAVCTcpRecvBuf@@@Z 004173fa f   xnetm:socktcp.obj
 0002:000052bc       ?TcpCompletePendingRecvReqFast@CXnSock@@AAEIPAVCTcpSocket@@EPAEI@Z 0041749c f   xnetm:socktcp.obj
 0002:00005329       ?TcpParseOptions@CXnSock@@AAEHPAVCTcpSocket@@PAUCTcpHdr@@PAU_TcpOptions@@@Z 00417509 f   xnetm:socktcp.obj
 0002:000053a9       ?TcpTrimBacklog@CXnSock@@AAEXPAVCTcpSocket@@I@Z 00417589 f   xnetm:socktcp.obj
 0002:000053f5       ?TcpListen@CXnSock@@AAEJPAVCTcpSocket@@H@Z 004175d5 f   xnetm:socktcp.obj
 0002:00005458       ?TcpCopyRecvData@CXnSock@@AAEIPAVCTcpSocket@@PAVCRecvReq@@@Z 00417638 f   xnetm:socktcp.obj
 0002:0000550b       ?TcpPacketAlloc@CXnSock@@AAEPAVCPacket@@PAVCTcpSocket@@UCIpAddr@@IIIP8CXnVoid@@AEXPAV2@@Z@Z 004176eb f   xnetm:socktcp.obj
 0002:0000553e       ?TcpPacketFree@CXnSock@@AAEXPAVCPacket@@@Z 0041771e f   xnetm:socktcp.obj
 0002:00005550       ?TcpSendSegment@CXnSock@@AAEXPAVCTcpSocket@@PAVCTcpSendBuf@@H@Z 00417730 f   xnetm:socktcp.obj
 0002:000056c9       ?EnqueueChild@CTcpSocket@@QAEXPAV1@@Z 004178a9 f   xnetm:socktcp.obj
 0002:00005733       ?GetConnectedChild@CTcpSocket@@QAEPAV1@XZ 00417913 f   xnetm:socktcp.obj
 0002:00005762       ?DequeueConnectedChild@CTcpSocket@@QAEPAV1@XZ 00417942 f   xnetm:socktcp.obj
 0002:0000577e       ?TcpReset@CXnSock@@AAEPAVCTcpSocket@@PAV2@J@Z 0041795e f   xnetm:socktcp.obj
 0002:000058d2       ?TcpCloneChild@CXnSock@@AAEPAVCTcpSocket@@PAV2@@Z 00417ab2 f   xnetm:socktcp.obj
 0002:00005902       ?TcpEmitRST@CXnSock@@AAEXPAVCTcpSocket@@UCIpAddr@@UCIpPort@@2KKE@Z 00417ae2 f   xnetm:socktcp.obj
 0002:000059c2       ?TcpResetPeer@CXnSock@@AAEXPAVCTcpSocket@@@Z 00417ba2 f   xnetm:socktcp.obj
 0002:000059f7       ?TcpEmitACK@CXnSock@@AAEXPAVCTcpSocket@@@Z 00417bd7 f   xnetm:socktcp.obj
 0002:00005ad8       ?TcpUpdatePersistFlag@CXnSock@@AAEHPAVCTcpSocket@@@Z 00417cb8 f   xnetm:socktcp.obj
 0002:00005b39       ?TcpDoFastRexmit@CXnSock@@AAEXPAVCTcpSocket@@@Z 00417d19 f   xnetm:socktcp.obj
 0002:00005ba7       ?TcpProcessFIN@CXnSock@@AAEXPAVCTcpSocket@@PAUCTcpHdr@@K@Z 00417d87 f   xnetm:socktcp.obj
 0002:00005c70       ?TcpConnectionEstablished@CXnSock@@AAEXPAVCTcpSocket@@PAUCTcpHdr@@@Z 00417e50 f   xnetm:socktcp.obj
 0002:00005dcc       ?TcpRead@CXnSock@@AAEJPAVCTcpSocket@@PAVCRecvReq@@@Z 00417fac f   xnetm:socktcp.obj
 0002:00005e89       ?TcpStartOutput@CXnSock@@AAEHPAVCTcpSocket@@@Z 00418069 f   xnetm:socktcp.obj
 0002:00005f80       ?TcpXmitTimeout@CXnSock@@AAEPAVCTcpSocket@@PAV2@@Z 00418160 f   xnetm:socktcp.obj
 0002:0000604f       ?TcpQueueSegment@CXnSock@@AAEXPAVCTcpSocket@@PAVCPacket@@EI@Z 0041822f f   xnetm:socktcp.obj
 0002:000060e7       ?TcpTimer@CXnSock@@AAEXPAVCTimer@@@Z 004182c7 f   xnetm:socktcp.obj
 0002:000061c4       ?TcpEmitSYN@CXnSock@@AAEJPAVCTcpSocket@@H@Z 004183a4 f   xnetm:socktcp.obj
 0002:0000629a       ?TcpEmitFIN@CXnSock@@AAEJPAVCTcpSocket@@@Z 0041847a f   xnetm:socktcp.obj
 0002:000062d5       ?TcpAcceptConnReqActive@CXnSock@@AAEHPAVCTcpSocket@@PAUCTcpHdr@@@Z 004184b5 f   xnetm:socktcp.obj
 0002:00006367       ?TcpShutdown@CXnSock@@AAEJPAVCTcpSocket@@KH@Z 00418547 f   xnetm:socktcp.obj
 0002:00006466       ?TcpSend@CXnSock@@AAEJPAVCTcpSocket@@PAVCSendReq@@I@Z 00418646 f   xnetm:socktcp.obj
 0002:000065fa       ?TcpUpdateSndUna@CXnSock@@AAEXPAVCTcpSocket@@K@Z 004187da f   xnetm:socktcp.obj
 0002:00006874       ?TcpRecvData@CXnSock@@AAEPAVCTcpSocket@@PAV2@PAUCTcpHdr@@PAEI@Z 00418a54 f   xnetm:socktcp.obj
 0002:00006ba2       ?TcpClose@CXnSock@@AAEHPAVCTcpSocket@@H@Z 00418d82 f   xnetm:socktcp.obj
 0002:00006c37       ?TcpConnect@CXnSock@@AAEJPAVCTcpSocket@@UCIpAddr@@UCIpPort@@H@Z 00418e17 f   xnetm:socktcp.obj
 0002:00006dfd       ?TcpAcceptConnReqPassive@CXnSock@@AAEHPAVCTcpSocket@@PAUCTcpHdr@@UCIpAddr@@@Z 00418fdd f   xnetm:socktcp.obj
 0002:00006ead       ?TcpRecv@CXnSock@@AAEXPAVCPacket@@PAUCIpHdr@@PAUCTcpHdr@@II@Z 0041908d f   xnetm:socktcp.obj
 0002:00007209       ?UdpShutdown@CXnSock@@AAEJPAVCSocket@@K@Z 004193e9 f   xnetm:sockudp.obj
 0002:0000726d       ?UdpRead@CXnSock@@AAEJPAVCSocket@@PAVCRecvReq@@@Z 0041944d f   xnetm:sockudp.obj
 0002:0000733a       ?UdpSend@CXnSock@@AAEJPAVCSocket@@PAVCSendReq@@I@Z 0041951a f   xnetm:sockudp.obj
 0002:000074d5       ?UdpConnect@CXnSock@@AAEJPAVCSocket@@UCIpAddr@@UCIpPort@@@Z 004196b5 f   xnetm:sockudp.obj
 0002:000075c9       ?UdpRecvData@CXnSock@@AAEXPAVCSocket@@UCIpAddr@@UCIpPort@@PAEI@Z 004197a9 f   xnetm:sockudp.obj
 0002:000076cc       ?UdpPacketFree@CXnSock@@AAEXPAVCPacket@@@Z 004198ac f   xnetm:sockudp.obj
 0002:0000774c       ?UdpRecv@CXnSock@@AAEXPAVCPacket@@PAUCIpHdr@@PAUCUdpHdr@@I@Z 0041992c f   xnetm:sockudp.obj
 0002:00007824       ?NicStartXmitRecv@CXnNic@@AAEXXZ 00419a04 f   xnetm:nicx.obj
 0002:0000784c       ?NicStopXmitRecv@CXnNic@@AAEXXZ 00419a2c f   xnetm:nicx.obj
 0002:000078bf       ?NicProcessIsr@CXnNic@@AAEEXZ 00419a9f f   xnetm:nicx.obj
 0002:000078d8       ?NicMiiInterrupt@CXnNic@@AAEXKH@Z 00419ab8 f   xnetm:nicx.obj
 0002:0000795e       ?NicXmitReady@CXnNic@@QAEHXZ 00419b3e f   xnetm:nicx.obj
 0002:00007980       ?NicStart@CXnNic@@IAEXXZ   00419b60 f   xnetm:nicx.obj
 0002:00007996       ?AttachClient@CXbdmServer@CXnNic@@UAEXPAVCXbdmClient@2@@Z 00419b76 f   xnetm:nicx.obj
 0002:000079b2       ?XmitReady@CXbdmServer@CXnNic@@UAEHXZ 00419b92 f   xnetm:nicx.obj
 0002:000079bd       ?GetXnAddr@CXbdmServer@CXnNic@@UAEKPAUXNADDRXBDM@2@@Z 00419b9d f   xnetm:nicx.obj
 0002:000079ec       ?NicGetOtherXnAddr@CXnNic@@QAEKPAUXNADDR@@@Z 00419bcc f   xnetm:nicx.obj
 0002:00007a45       ?NicIsr@CXnNic@@CGEPAU_KINTERRUPT@@PAX@Z 00419c25 f   xnetm:nicx.obj
 0002:00007a51       ?NicRecvInterrupt@CXnNic@@AAEXXZ 00419c31 f   xnetm:nicx.obj
 0002:00007c11       ?NicXmitInterrupt@CXnNic@@AAEXXZ 00419df1 f   xnetm:nicx.obj
 0002:00007d17       ?NicXmit@CXnNic@@QAEXPAVCPacket@@@Z 00419ef7 f   xnetm:nicx.obj
 0002:00007e01       ?NicTimer@CXnNic@@QAEXXZ   00419fe1 f   xnetm:nicx.obj
 0002:00007e26       ?NicFlush@CXnNic@@IAEXXZ   0041a006 f   xnetm:nicx.obj
 0002:00007e68       ?NicStop@CXnNic@@IAEXXZ    0041a048 f   xnetm:nicx.obj
 0002:00007ec2       ?NicTerm@CXnNic@@IAEXXZ    0041a0a2 f   xnetm:nicx.obj
 0002:00007f63       ?HalShutdownNotification@CXnNic@@CGXPAU_HAL_SHUTDOWN_REGISTRATION@@@Z 0041a143 f   xnetm:nicx.obj
 0002:00007f9b       ?NicStop@CXbdmServer@CXnNic@@UAEXXZ 0041a17b f   xnetm:nicx.obj
 0002:00007fd1       ?InitClient@CXbdmServer@CXnNic@@UAEJIIPAUCEnetAddr@@PAH@Z 0041a1b1 f   xnetm:nicx.obj
 0002:00007ff3       ?DetachClient@CXbdmServer@CXnNic@@UAEXXZ 0041a1d3 f   xnetm:nicx.obj
 0002:00008027       ?Xmit@CXbdmServer@CXnNic@@UAEXPAX0I@Z 0041a207 f   xnetm:nicx.obj
 0002:0000806e       ?NicProcessDpc@CXnNic@@AAEXXZ 0041a24e f   xnetm:nicx.obj
 0002:000080ca       ?NicDpc@CXnNic@@CGXPAU_KDPC@@PAX11@Z 0041a2aa f   xnetm:nicx.obj
 0002:000080d6       ?NicInit@CXnNic@@IAEJPAUXNetInitParams@@@Z 0041a2b6 f   xnetm:nicx.obj
 0002:000085be       _XNetOpenConfigVolume@0    0041a79e f   xnetm:xnetp.obj
 0002:0000860c       _XNetLoadConfigSector@16   0041a7ec f   xnetm:xnetp.obj
 0002:00008691       _XNetCloseConfigVolume@4   0041a871 f   xnetm:xnetp.obj
 0002:000086a8       _XConfigChecksum@8         0041a888 f i xnetm:xnetp.obj
 0002:000086d2       _XNetSaveConfigSector@16   0041a8b2 f   xnetm:xnetp.obj
 0002:0000876f       ?ActiveDhcpAddr@CXnIp@@AAEHXZ 0041a94f f   xnetm:ipdhcp.obj
 0002:0000877b       ?ActiveAutonetAddr@CXnIp@@AAEHXZ 0041a95b f   xnetm:ipdhcp.obj
 0002:00008787       ?ActiveStaticAddr@CXnIp@@AAEHXZ 0041a967 f   xnetm:ipdhcp.obj
 0002:00008794       ?ActiveNoAddr@CXnIp@@AAEHXZ 0041a974 f   xnetm:ipdhcp.obj
 0002:000087a0       ?DhcpTerm@CXnIp@@AAEXXZ    0041a980 f   xnetm:ipdhcp.obj
 0002:000087af       ?DhcpTime@CXnIp@@AAEKXZ    0041a98f f   xnetm:ipdhcp.obj
 0002:000087d7       ?DhcpAppendParamReqList@@YGPAEPAE@Z 0041a9b7 f   xnetm:ipdhcp.obj
 0002:000087f6       ?DhcpComputeSecsSinceStart@CXnIp@@AAEXXZ 0041a9d6 f   xnetm:ipdhcp.obj
 0002:0000881b       ?DhcpTimerSetRelative@CXnIp@@AAEXII@Z 0041a9fb f   xnetm:ipdhcp.obj
 0002:00008854       ?DhcpTimerSetAbsolute@CXnIp@@AAEXK@Z 0041aa34 f   xnetm:ipdhcp.obj
 0002:0000889a       ?DhcpComputeTimeout@CXnIp@@AAEXXZ 0041aa7a f   xnetm:ipdhcp.obj
 0002:0000896d       ?DhcpResetInterface@CXnIp@@AAEXXZ 0041ab4d f   xnetm:ipdhcp.obj
 0002:0000899a       ?DhcpSendMessage@CXnIp@@AAEJPAVCPacket@@IH@Z 0041ab7a f   xnetm:ipdhcp.obj
 0002:00008a1b       ?DhcpAppendLeaseTimeOption@CXnIp@@AAEPAEPAE@Z 0041abfb f   xnetm:ipdhcp.obj
 0002:00008a69       ?DhcpFillMessageHeader@CXnIp@@AAEPAEPAEH@Z 0041ac49 f   xnetm:ipdhcp.obj
 0002:00008b1e       ?DhcpSendDiscover@CXnIp@@AAEJXZ 0041acfe f   xnetm:ipdhcp.obj
 0002:00008ba1       ?DhcpSendRequest@CXnIp@@AAEJXZ 0041ad81 f   xnetm:ipdhcp.obj
 0002:00008c6e       ?DhcpValidateOffer@CXnIp@@AAEHUCIpAddr@@PAUCDhcpOptions@1@@Z 0041ae4e f   xnetm:ipdhcp.obj
 0002:00008cfe       ?DhcpAddOrRemoveGateways@CXnIp@@AAEXH@Z 0041aede f   xnetm:ipdhcp.obj
 0002:00008d62       ?DhcpSetDefaultGateways@CXnIp@@AAEXXZ 0041af42 f   xnetm:ipdhcp.obj
 0002:00008d81       ?DhcpUseOptionParams@CXnIp@@AAEXPAUCDhcpOptions@1@@Z 0041af61 f   xnetm:ipdhcp.obj
 0002:00008ea9       ?DhcpParseOptionParams@CXnIp@@AAEJPAUCDhcpOptions@1@PBEIPAE@Z 0041b089 f   xnetm:ipdhcp.obj
 0002:0000909f       ?DhcpChangeState@CXnIp@@AAEXH@Z 0041b27f f   xnetm:ipdhcp.obj
 0002:00009174       ?DhcpProcessOffer@CXnIp@@AAEJUCIpAddr@@PAUCDhcpOptions@1@@Z 0041b354 f   xnetm:ipdhcp.obj
 0002:000091b3       ?DhcpProcessAck@CXnIp@@AAEJUCIpAddr@@PAUCDhcpOptions@1@@Z 0041b393 f   xnetm:ipdhcp.obj
 0002:00009251       ?DhcpProcessNak@CXnIp@@AAEJUCIpAddr@@@Z 0041b431 f   xnetm:ipdhcp.obj
 0002:00009271       ?DhcpSelectAutonetAddr@CXnIp@@AAEXXZ 0041b451 f   xnetm:ipdhcp.obj
 0002:000092fe       ?DhcpConfig@CXnIp@@AAEHPBUXNetConfigParams@@@Z 0041b4de f   xnetm:ipdhcp.obj
 0002:00009442       ?DhcpRecv@CXnIp@@AAEXPAVCPacket@@PAUCUdpHdr@@I@Z 0041b622 f   xnetm:ipdhcp.obj
 0002:000095ca       ?DhcpNotifyAddressConflict@CXnIp@@AAEXXZ 0041b7aa f   xnetm:ipdhcp.obj
 0002:000095d9       ?DhcpTimer@CXnIp@@AAEXPAVCTimer@@@Z 0041b7b9 f   xnetm:ipdhcp.obj
 0002:00009715       ?IpRecvArp@CXnIp@@IAEXPAUCEnetAddr@@@Z 0041b8f5 f   xnetm:ipdhcp.obj
 0002:0000971d       ?DhcpInit@CXnIp@@AAEJXZ    0041b8fd f   xnetm:ipdhcp.obj
 0002:0000974a       ?EnetQueuePush@CXnEnet@@IAEXXZ 0041b92a f   xnetm:enet.obj
 0002:0000975c       ?EnetXmit@CXnEnet@@QAEXPAVCPacket@@UCIpAddr@@@Z 0041b93c f   xnetm:enet.obj
 0002:0000979c       ?EnetStop@CXnEnet@@IAEXXZ  0041b97c f   xnetm:enet.obj
 0002:000097be       ?ArpXmit@CXnEnet@@AAEXGUCIpAddr@@0PAUCEnetAddr@@@Z 0041b99e f   xnetm:enet.obj
 0002:0000986e       ?ArpLookup@CXnEnet@@AAEPAUCArpEntry@1@UCIpAddr@@W4ArpResolve@1@@Z 0041ba4e f   xnetm:enet.obj
 0002:00009957       ?ArpTimer@CXnEnet@@AAEXPAVCTimer@@@Z 0041bb37 f   xnetm:enet.obj
 0002:00009a0a       ?ArpRecv@CXnEnet@@AAEXPAVCPacket@@@Z 0041bbea f   xnetm:enet.obj
 0002:00009b93       ?EnetFillAndXmit@CXnEnet@@AAEXPAVCPacket@@PAUCEnetAddr@@@Z 0041bd73 f   xnetm:enet.obj
 0002:00009bc4       ?EnetTerm@CXnEnet@@IAEXXZ  0041bda4 f   xnetm:enet.obj
 0002:00009c34       ?EnetXmitArp@CXnEnet@@QAEXUCIpAddr@@@Z 0041be14 f   xnetm:enet.obj
 0002:00009c53       ?EnetRecv@CXnEnet@@IAEXPAVCPacket@@I@Z 0041be33 f   xnetm:enet.obj
 0002:00009c80       ?EnetPush@CXnEnet@@QAEXXZ  0041be60 f   xnetm:enet.obj
 0002:00009d71       ?EnetDpc@CXnEnet@@CGXPAU_KDPC@@PAX11@Z 0041bf51 f   xnetm:enet.obj
 0002:00009d7d       ?EnetInit@CXnEnet@@IAEJPAUXNetInitParams@@@Z 0041bf5d f   xnetm:enet.obj
 0002:00009de4       _tcpipxsum@12              0041bfc4 f   xnetm:tcpipxsum.obj
 0002:00009f20       ?IcmpRecv@CXnIp@@AAEXPAVCPacket@@PAUCIpHdr@@PAXI@Z 0041c100 f   xnetm:ipicmp.obj
 0002:0000a068       _g_abOakleyGroup1Mod       0041c248     xnetm:base.obj
 0002:0000a0c8       _g_abOakleyGroup1Base      0041c2a8     xnetm:base.obj
 0002:0000a128       ?s_XNetParamsDef@CXnBase@@0UXNetParams@@B 0041c308     xnetm:base.obj
 0002:0000a158       ?s_XNetParamsMin@CXnBase@@0UXNetParams@@B 0041c338     xnetm:base.obj
 0002:0000a188       ?s_XNetParamsMax@CXnBase@@0UXNetParams@@B 0041c368     xnetm:base.obj
 0002:0000a1b8       ?_abPktTypeInfo@CPacket@@2QBEB 0041c398     xnetm:base.obj
 0002:0000a1d0       ??_C@_0BN@OGMPKPAN@?2Device?2Harddisk0?2partition0?$AA@ 0041c3b0     xnetm:xnetp.obj
 0003:00000000       _hsrAPIC                   0041c3e0     dminit.obj
 0003:00000010       _szIniName                 0041c3f0     dminit.obj
 0003:0000001c       _szDxtDir                  0041c3fc     dminit.obj
 0003:00000024       _oszDxtTemplate            0041c404     dminit.obj
 0003:00000030       _portcounter               0041c410     dmserv.obj
 0003:00000034       _ostDashBuffer             0041c414     dmserv.obj
 0003:00000060       _ostDash                   0041c440     dmserv.obj
 0003:00000068       _XdkLauncherPathname       0041c448     dmserv.obj
 0003:00000118       _rgchh                     0041c4f8     dmserv.obj
 0003:000006b8       _cchh                      0041ca98     dmserv.obj
 0003:000006f8       _fAllowKd                  0041cad8     dmnotify.obj
 0003:000006fc       _rgszExec                  0041cadc     dmnotify.obj
 0003:0000070c       _rgfsub                    0041caec     dmmodule.obj
 0003:00000724       _obtCounter                0041cb04     dmcount.obj
 0003:00000740       _rgszMemCounters           0041cb20     dmcount.obj
 0003:00000758       _rggcGPU                   0041cb38     dmcount.obj
 0003:00000788       _obtPob                    0041cb68     dmprofil.obj
 0003:000007a4       _lePobHead                 0041cb84     dmprofil.obj
 0003:000007ac       _rgulIntervalTable         0041cb8c     dmprofil.obj
 0003:000007e8       _DriveNameConversionTable  0041cbc8     dmfile.obj
 0003:000008a8       __FlashDeviceClass         0041cc88     flash.obj
 0003:000008c8       _FlashSizeMap              0041cca8     flash.obj
 0003:000008e0       _g_rgdwLoc                 0041ccc0     dmxapi:compstra.obj
 0003:00000d10       _MmHeapSegmentReserve      0041d0f0     xapirtl:heap.obj
 0003:00000d14       _MmHeapSegmentCommit       0041d0f4     xapirtl:heap.obj
 0003:00000d18       _MmHeapDeCommitTotalFreeThreshold 0041d0f8     xapirtl:heap.obj
 0003:00000d1c       _MmHeapDeCommitFreeBlockThreshold 0041d0fc     xapirtl:heap.obj
 0003:00000d20       __NLG_Destination          0041d100     libcntpr:exsup.obj
 0003:00000d30       __fltused                  0041d110     libcntpr:stubs.obj
 0003:00000d34       __ldused                   0041d114     libcntpr:stubs.obj
 0003:00000f90       ?g_lXnLock@@3JA            0041d370     xnetm:xnet.obj
 0003:00000f94       ?g_pXn@@3PAVCXn@@A         0041d374     xnetm:xnet.obj
 0003:00000f98       ___@@_PchSym_@00@UcylcUkirezgvUmglhUmvgUorynUlyqUrDIGUcmkOlyq@xnetm 0041d378     xnetm:xnp.obj
 0003:00000fa0       ?s_InterruptObject@CXnNic@@0U_KINTERRUPT@@A 0041d380     xnetm:nicx.obj
 0003:00001010       ___fastflag                0041d3f0     libcntpr:stubs.obj
 0003:00001014       _KernelRomBase             0041d3f4     <common>
 0003:00001018       _DmProfileData             0041d3f8     <common>
 0003:0000101c       _DmProfileSavedCtxSwapNotify 0041d3fc     <common>
 0003:00001020       _ExpSmallDmPoolLookasideLists 0041d400     <common>
 0003:000010e0       _ExpTaggedPoolLock         0041d4c0     <common>
 0003:000010e4       _PoolBigPageTable          0041d4c4     <common>
 0003:000010e8       _PoolTrackTableMask        0041d4c8     <common>
 0003:000010ec       _PoolTrackTableSize        0041d4cc     <common>
 0003:000010f0       _PoolBigPageTableHash      0041d4d0     <common>
 0003:000010f4       _FirstPrint                0041d4d4     <common>
 0003:00001100       _DmPoolDescriptor          0041d4e0     <common>
 0003:00001510       _PoolTrackTable            0041d8f0     <common>
 0003:00001514       _PoolBigPageTableSize      0041d8f4     <common>
 0003:00001518       _g_fResetInterval          0041d8f8     <common>
 0003:0000151c       _ulNextProfInt             0041d8fc     <common>
 0003:00001520       _ulCurProfBase             0041d900     <common>
 0003:00001524       _hpobGPU                   0041d904     <common>
 0003:00001540       _tmrRefreshCounters        0041d920     <common>
 0003:00001580       _rgulSystemTimes           0041d960     <common>
 0003:00001598       _hCounterDir               0041d978     <common>
 0003:000015a0       _rgulPages                 0041d980     <common>
 0003:000015c0       _rgleUpdateQueues          0041d9a0     <common>
 0003:00001620       _dpcRefreshCounters        0041da00     <common>
 0003:0000163c       _ileCur                    0041da1c     <common>
 0003:00001640       _csLoader                  0041da20     <common>
 0003:0000165c       _pbplRoot                  0041da3c     <common>
 0003:00001660       _fHaltAllThreads           0041da40     <common>
 0003:00001680       _csBplScratch              0041da60     <common>
 0003:0000169c       _pbplTrace                 0041da7c     <common>
 0003:000016a0       _rghwbp                    0041da80     <common>
 0003:000016c0       _pbplScratch               0041daa0     <common>
 0003:000016c4       _iBreakTrace               0041daa4     <common>
 0003:000016e0       _csHwBps                   0041dac0     <common>
 0003:000016fc       _dwExecState               0041dadc     <common>
 0003:00001700       _dpcBreakIn                0041dae0     <common>
 0003:00001720       _ctxDF                     0041db00     <common>
 0003:00001958       _fUsingSessionList         0041dd38     <common>
 0003:0000195c       _psessFirst                0041dd3c     <common>
 0003:00001960       _rgnnPersist               0041dd40     <common>
 0003:000019c0       _rgbDFStack                0041dda0     <common>
 0003:000029c0       _g_ppdfnNext               0041eda0     <common>
 0003:000029c4       _g_pdfnFirst               0041eda4     <common>
 0003:000029c8       _psessFree                 0041eda8     <common>
 0003:000029cc       _fPruneList                0041edac     <common>
 0003:000029e0       _csNotifySockList          0041edc0     <common>
 0003:000029fc       _g_grbitStopOn             0041eddc     <common>
 0003:00002a00       _csNotify                  0041ede0     <common>
 0003:00002a20       _evtNotifyList             0041ee00     <common>
 0003:00002a30       _pfnKdpTrap                0041ee10     <common>
 0003:00002a40       _rgsockNotify              0041ee20     <common>
 0003:00002a60       _g_fAdminPasswd            0041ee40     <common>
 0003:00002a68       _g_luAdminPasswd           0041ee48     <common>
 0003:00002a80       _csUserList                0041ee60     <common>
 0003:00002aa0       _csAccept                  0041ee80     <common>
 0003:00002ac0       _g_luBoxId                 0041eea0     <common>
 0003:00002ae0       _rgcst                     0041eec0     <common>
 0003:000034c0       _g_fServShutdown           0041f8a0     <common>
 0003:000034e0       _rgpech                    0041f8c0     <common>
 0003:00003520       _rgchDbgName               0041f900     <common>
 0003:00003620       _g_fDebugging              0041fa00     <common>
 0003:00003630       _kevtServ                  0041fa10     <common>
 0003:00003640       _csEch                     0041fa20     <common>
 0003:0000365c       _g_fLockLevel              0041fa3c     <common>
 0003:00003660       _pthrServ                  0041fa40     <common>
 0003:00003664       _g_fDebugSecureMode        0041fa44     <common>
 0003:00003680       _csIniFile                 0041fa60     <common>
 0003:0000369c       _fBootWait                 0041fa7c     <common>
 0003:000036a0       _pszCmdLine                0041fa80     <common>
 0003:000036c0       _rgchTitleDir              0041faa0     <common>
 0003:00003810       _kevtNull                  0041fbf0     <common>
 0003:00003820       _g_dmi                     0041fc00     <common>
 0003:0000385c       _pprocSystem               0041fc3c     <common>
 0003:00003860       _g_dmgd                    0041fc40     <common>
 0003:00003880       _g_dmxapi                  0041fc60     <common>
 0003:0000388c       _g_ulDbgIP                 0041fc6c     <common>
 0003:00003890       _g_fFinishedLoadingIniFile 0041fc70     <common>
 0003:000038a0       _rgchTitleName             0041fc80     <common>
 0003:000038e0       _g_hIniFile                0041fcc0     <common>
 0003:000038e4       _NtGlobalFlag              0041fcc4     <common>
 0003:000038e8       _errno                     0041fcc8     <common>
 0004:00000000       _XapiLastErrorCode         0041fce0     dmxapi:error.obj
 0006:00000000       __IMPORT_DESCRIPTOR_xboxkrnl 0041fe60     xboxkrnl:xboxkrnl.exe
 0006:00000014       __NULL_IMPORT_DESCRIPTOR   0041fe74     xboxkrnl:xboxkrnl.exe
 0007:00000000       _XapiBuildNumber           004200a0     dmxapi:basedll.obj
 0007:00000010       _XNetBuildNumberM          004200b0     xnetm:sock.obj
 0007:00000020       _XboxKrnlBuildNumber       004200c0     xboxkrnl:bldnum.obj

 entry point at        0001:00002aca

 Static symbols

 0001:0000d793       _HrGetFrameCount@8         0040daf3 f   dmcount.obj
 0001:000111c0       _$$$00001                  00411520 f   libcntpr:strchr.obj
 0001:000113b8       $$$00003                   00411718 f   libcntpr:exsup3.obj
 0001:000114a9       _write_char                00411809 f   libcntpr:output.obj
 0001:000114dc       _write_multi_char          0041183c f   libcntpr:output.obj
 0001:00011500       _write_string              00411860 f   libcntpr:output.obj
 0001:00011ba0       $$$00001                   00411f00 f   libcntpr:exsup.obj
 0001:00011bc0       __unwind_handler           00411f20 f   libcntpr:exsup.obj
 0001:00011bc0       $$$00003                   00411f20 f   libcntpr:exsup.obj
 0001:00011be2       $$$00005                   00411f42 f   libcntpr:exsup.obj
 0001:00011c4a       $$$00007                   00411faa f   libcntpr:exsup.obj
 0001:00011c8e       $$$00011                   00411fee f   libcntpr:exsup.obj
 0002:00002b5c       ?QueryTsc@@YGXPAT_LARGE_INTEGER@@@Z 00414d3c f   xnetm:halx.obj
